:1080000000000120290C0100A5E30000A5E3000009
:10801000A5E30000A5E30000A5E3000000000000C8
:10802000000000000000000000000000A5E30000C8
:10803000A5E3000000000000A5E300001D8600008D
:10804000A5E30000A5E30000A5E30000A5E3000010
:10805000A5E30000A5E30000A5E30000A5E3000000
:10806000A5E30000A5E30000A5E30000A5E30000F0
:10807000A5E30000A5E30000A5E30000A5E30000E0
:10808000A5E30000A5E30000A5E30000A5E30000D0
:10809000A5E30000A5E30000A5E30000A5E30000C0
:1080A000A5E30000BDD50000A5E30000A5E30000A6
:1080B000A5E30000A5E30000A5E30000A5E30000A0
:1080C000A5E30000A5E30000A5E30000A5E3000090
:1080D000A5E30000A5E30000A5E30000D1D1000066
:1080E000A5E30000A5E30000A5E30000A5E3000070
:1080F000A5E30000A5E30000A5E30000A5E3000060
:10810000A5E30000A5E30000A5E30000A5E300004F
:10811000A5E30000C1F50000A5E30000A5E3000011
:10812000A5E30000A5E30000A5E30000A5E300002F
:10813000A5E30000A5E30000A5E30000A5E300001F
:10814000A5E30000A5E3000071870000A5E300009F
:10815000A5E30000A5E30000A5E30000A5E30000FF
:10816000A5E300000DD20000A5E30000A5E3000098
:10817000A5E30000A5E30000A5E30000A5E30000DF
:08818000A5E30000A5E30000E7
:10840000FFFFFFFFFFFFFFFFFFFFFFFF7EF9FFFF03
:1084100010B5054C237833B9044B13B10448AFF3BE
:1084200000800123237010BD0086FF1F00000000A4
:10843000041401000C4B43B10C480D4910B5AFF3C7
:1084400000800C48036823B910BD0A48036833B99B
:108450007047094B002BF7D0BDE810401847064B7A
:10846000002BF5D0184700BF0000000004140100E5
:108470000486FF1F6C85FF1F0000000080F3118839
:1084800070472F4B41F238015A5842F478525A50F3
:108490002C4A927902F00C020C2A4FD041F244028D
:1084A0002949995003F558339A78110748BF9A78AB
:1084B000264944BF42F008029A70214B41F244021F
:1084C000995041F204015A5842F4803242F0C002FD
:1084D0005A501A6842F440221A6003F5E833242205
:1084E0005A701B4A80211170A2221A70DA7802F0A9
:1084F0001F02DA7003221A7100225A719A799207C8
:10850000FCD59A79D006FCD40E4B19469A7902F024
:108510000C02082AFAD140225A718B7903F00C031D
:10852000082BFAD1074B1A4699794906FCD5222126
:108530001970937903F00C030C2BFAD1704700BF2C
:1085400000700440004006400000330100001301A9
:10855000005006402B4B5A7902F0E0025A711A790A
:1085600002F0F8021A71284A136843F004031360FA
:10857000264A136823F0784323F001031360244B49
:108580001A7802F08C0242F050021A705A7802F007
:108590009C0242F040025A709A7802F0E6029A7009
:1085A0001C4A0023137083F311881B4B012283F8AC
:1085B000182383F81923022283F83C2383F83D23F0
:1085C00083F84B2383F84C2383F84D2383F84E2301
:1085D00083F84F23032283F81F2383F8212383F892
:1085E000232383F8252383F84223042283F82723B7
:1085F000052283F84923062283F83B23072283F8C8
:108600003523704700F007404080044000D0004010
:1086100000D0074000E0074000E100E00C4A13688A
:10862000013313600B4A1368013313600A4B1A6855
:108630003AB11A68013A1A601B6813B9074B012254
:108640001A70074B1A6812B11A68013A1A6070471B
:108650001C86FF1FF00500202403002020030020BB
:1086600028030020024B034A5A6007221A60704711
:1086700010E000E000770100014B1868704700BF70
:108680001C86FF1F1449154B41F22802072888BF9A
:10869000002010B553F82030114CB4FBF3F48B5884
:1086A00043F480638B500F4B4FF440729A63422027
:1086B000DA6305F095FE0C4B0022DA709A709A711D
:1086C000DA725A71C4F30422E4B21A705C70DA7878
:1086D00042F02C02DA7010BD00700440C811010095
:1086E000C0C62D0000B0044000A00E40094A136827
:1086F00051680133202B08BF00238B4208D011683A
:10870000114408721360044AD37843F08003D37095
:10871000704700BF2086FF1F00A00E400A4B996AD9
:10872000DA6A91420DD09A6A511C1A44996292F801
:10873000302002709A6A202A01D100229A62012018
:1087400070470020704700BF2086FF1F044B1A7837
:1087500002F0FF0012B100221A700120704700BF22
:1087600020030020014B1865704700BF2086FF1FC3
:1087700030B526480179C9B28C0617D5244BDA6A80
:108780009C6A0132202A08BF0022A2421BBFDC6A79
:10879000C579C27918191EBFEDB280F83050DA627F
:1087A0001C4A052010601A6D1B4B1A604A0608D53A
:1087B0001A4B4FF480529A60144AD37803F0BF03E7
:1087C000D3700B061BD5144B1868C0B9104B196831
:1087D0005A68914214D0114A4FF4805151605A683E
:1087E000511C1A445960117A084AC9B2D1715968AA
:1087F000202908BF5860D37843F04003D37030BDC0
:10880000024AD37803F07F03F8E700BF00A00E40D0
:108810002086FF1F240300202803002080F00F4043
:1088200062B67047FFF7FCBF72B67047FFF7FCBF38
:108830004FF0E02318B1034AC3F80C2D7047024AE9
:10884000FAE700BF0400FA050100FA05F7B544484D
:10885000444C454D454E4FF480731622436083606F
:108860000361A2601E226261414A53629364D36431
:108870001365536593654FF400226A61AA603D4A0F
:108880004FF4907151621363936402F53422803285
:108890004FF4905191604FF48021516001F5905157
:1088A0005161354A40F20311116051609160D1600D
:1088B000116151619161D161304900224A613049B1
:1088C0000B614B618B618B6601F5322101F5807183
:1088D0008E604E6103600826C360134611460A206D
:1088E0002A46B4461F46A646C4F804C00197019D17
:1088F000B5F57A7F2AD3DEF81050A660ED0748BFA1
:1089000001310197019DB5F57A7F23D3DEF8105030
:10891000ED0758BF01330138E6D10A2919491DD1A5
:108920000A2B1BD101230B700D4B4FF4E061196032
:10893000D96003F580534FF48071196001235360AF
:10894000536943F00103536103B0F0BD019D01354C
:108950000195CCE7019D01350195D3E70023E2E7BE
:108960000090044000F00F4040F00F407000000401
:1089700000A0044000B0044000C00440C0F00F401C
:1089800000D0044060030020F7B5104B1B78D3B132
:108990000F4B104D02210F46042000241E469F60FD
:1089A00058600194019AAA4209D97160B06001949B
:1089B000019AAA42F3D8019A01320192F8E7019A8A
:1089C00001320192EEE703B0F0BD00BF600300206A
:1089D00000F00F401FA10700032806D8DFE800F0D1
:1089E0000206080A1022054B5A6070472022FAE757
:1089F0004022F8E74FF08062F5E700BF00F10F403A
:108A0000032806D8DFE800F00206080A1022054B0A
:108A10009A6070472022FAE74022F8E74FF0806220
:108A2000F5E700BF00F10F4010B50021044644FAFD
:108A300001F3DB07C8B205D5FFF7CEFF01310829E6
:108A4000F5D110BDFFF7DCFFF8E708B5032813D810
:108A5000DFE800F0020C0E10002004F03DFC43F2B1
:108A60007C03984294BF0020012008BD0120F4E758
:108A70000220F2E70320F0E7002008BD032817D802
:108A8000DFE800F002070C110A4B1868C0F3001071
:108A90007047084B1868C0F340107047054B1868C2
:108AA000C0F380107047034B1868C0F380607047B4
:108AB0000020704700F10F4070B5002425460126C4
:108AC000E0B2FFF7C2FF18B106FA04F31D43EDB29E
:108AD0000134082CF4D1284670BD024B1869C043FC
:108AE000C0B27047C0F00F4037B50446FFF7C4FD71
:108AF0000546FFF7C1FD401B0028B8BF40420128D2
:108B0000F7DD0020012C8DF804008DF8050010D051
:108B100007D3022C11D0030648BF60F0FF0003B05A
:108B200030BD022201A9902004F004FE9DF804004B
:108B3000F1E7022201A99220F6E7224601A994203A
:108B4000F2E708B5082004F0C7FB5E2811D9134BE3
:108B50001A780AB901221A70082004F0BDFBA9286E
:108B60000FD90F4B1B7863B90E4B4FF400725A604C
:108B700008BD082004F0B0FB5428EDD80022074BB4
:108B8000E9E7082004F0A8FB952802D9044B1B78DC
:108B90001BB1044B4FF400729A6008BD7486FF1F2E
:108BA0004B03002080F00F40034B18780138012858
:108BB0008CBF0020012070477486FF1F034B18787C
:108BC000012806BF02221A70002070477486FF1F1A
:108BD000C0B205F021BBC0B205F00CBB08B507F070
:108BE00013FB05F0D1FD05F081FDBDE8084007F05D
:108BF0008DBB38B5054605F0CFFC08280AD90024FE
:108C00002819013405F048FD092CF9D105F078FD4B
:108C1000012038BD002038BD092105F0DDBC002051
:108C200005F06ABF2249234841F23C028B5843F4C5
:108C300040538B50204B012119601A6802431A607F
:108C40001E4ADA601A61DA6A42F08052DA621A6801
:108C500022F001021A601A6822F000621A60184AB3
:108C60004FF40073136053609360D36013615361DA
:108C70009361D361A2F5F032116011680143116074
:108C80001049D16001F520011161D16A41F0805194
:108C9000D162116821F001011160116821F00061B9
:108CA000116002F5E8329362D36213645364704733
:108CB00000700440000C1F8000C002400300013E11
:108CC00000B004400400513EFF2810B54FEA0043B5
:108CD00023D82B4C03F47C138AB141F000610B4381
:108CE0006363E36A002BFCDA254BDA6AD000FCD51B
:108CF000986BDA6A42F01042C0B2DA6210BD41F0FD
:108D000000410B436363E36A002BFCDAA06BE36A68
:108D100043F01043C0B2E36210BDB0F5007F17D23C
:108D2000184C03F47C135AB141F000610B436363A8
:108D3000E36A002BFCDA134BDA6AD100FCD5D7E7E3
:108D400041F000410B436363E36A002BFCDADDE78B
:108D50000D4C03F47C135AB141F000610B43636383
:108D6000E36A002BFCDA084BDA6AD200FCD5BFE7D5
:108D700041F000410B436363E36A002BFCDAC5E773
:108D800000C0024000D0024000C00A4010B5FFF70A
:108D900073FC0446FFF770FC001B0028B8BF40427C
:108DA0000628F7DD10BD07B5030A8DF805008DF81C
:108DB0000610032201A9A0208DF8043004F094FCD1
:108DC000FFF7E4FF03B05DF804FBF0B515460022A1
:108DD0008BB00F461446AC4201D10BB0F0BD0AABCC
:108DE0001344395D03F8221C531CC618F10602D047
:108DF000691E8C420DD1030A8DF80500033201A9CA
:108E0000A0208DF8043004F06FFCFFF7BFFF304660
:108E1000002301341A46DEE71FB5030A8DF80C3033
:108E2000022203AB8DF80D0000921946A02004F039
:108E3000A7FC9DF80C0005B05DF804FB1FB5030A04
:108E40008DF80C308DF80D0000920B46022203A91C
:108E5000A02004F095FC05B05DF804FB30B4C0EB35
:108E6000C000074C0D68255022188C8894808B799F
:108E7000937100F5B040072230BCFFF7A6BF00BFDA
:108E80007586FF1F054BC0EBC000184403680B60DC
:108E900083888B8083798B71704700BF7586FF1F35
:108EA00030B500238BB001AD1A465A550133222B41
:108EB000FBD14FF4B044230A8DF805402222294605
:108EC000A02020348DF8043004F00EFCFFF75EFF84
:108ED000B4F5484FEFD10B4900220C461346C2EBC4
:108EE000C20020440132B2F5805F0B704B708B7072
:108EF000C37003714371837101F10701EFD10BB0AE
:108F000030BD00BF7586FF1F13B50C46C0EBC00017
:108F10000722694600F5B040FFF790FF9DF800205A
:108F200023789A4212D19DF8012063789A420DD19C
:108F30009DF80220A3789A4208D1DDF80300D4F806
:108F40000330C31A5842584102B010BD0020FBE75D
:108F500070477FB545F2FF70FFF75EFF552803D1DC
:108F6000334B1B78002B3DD0002145F2FF70FFF7FB
:108F70001AFFFFF795FF40222E490020FFF725FF3B
:108F8000402210462C49FFF720FF40222A4980202A
:108F9000FFF71BFF04AD40222749C020FFF715FF54
:108FA000002345F8043D4FF4D36440F6780620468C
:108FB000042229460434FFF708FFB442F7D1002306
:108FC00003934FF4FF6440F6D80620460422294656
:108FD0000434FFF7FAFEB442F7D1552145F2FF7091
:108FE000FFF7E1FE402213490020FFF727FF402250
:108FF00010461249FFF722FF402211498020FFF757
:109000001DFF40220F49C020FFF718FF58238DF89D
:10901000083000238DF809304FF4E043009302221A
:10902000094B02A9A02004F0ABFB04B070BD00BF47
:10903000600300200C80FF1FF8110100780300205E
:10904000B8030020F80300207586FF1F0000000011
:10905000044B9B78022B044B8CBF042203221A7012
:10906000704700BFD8040020F405002073B5CB4D35
:109070006A78A52A2C4600F0708300F2AF80142A8B
:1090800000F03C8247D80C2A00F0EC8120D8042A5A
:1090900000F0AA8109D8012A00F07681C0F06F8122
:1090A000022A00F08781032266E1062A00F0C781C8
:1090B000C0F0B281072AF6D11021A87804F0D6FCBE
:1090C000EA780346D208A8780192C3F30722C0E1E8
:1090D000102A00F0F4810FD80E2A00F0E28140F24D
:1090E000D181AD78AE4BD4F8030003EB85039B69C7
:1090F00098472421024675E1122AA94B00F0F48119
:1091000040F2E881AD78D4F8030053F82530984751
:109110002321024666E11C2A00F03F8220D8182A4B
:1091200000F010820ED8162A00F0F68140F2F0818D
:10913000AD789B4BD4F8030053F825309847332182
:1091400002464FE11A2A00F01B8240F20A82D5F84B
:109150000310A878C9B202B0BDE8704004F064BD45
:109160007F2A00F0438216D8202A00F01F82212A8D
:1091700000F02D821F2A96D11021A87804F076FCE9
:10918000EB780246D1B2C2F30722A878019100928F
:1091900003F00F0360E1A22A00F0CD820FD88C2AE1
:1091A00081D1D5F80310A878C1F10801C9B204F043
:1091B00017FDA87802B0BDE8704004F01DBBA32ADB
:1091C00000F0C282A42A7FF46EAFD5F80310A8780D
:1091D000C9B202B0BDE8704004F06EBDBB2A00F019
:1091E000448371D8AD2A00F004831FD8A92A00F067
:1091F000E5820DD8A72A00F0D88240F2C282D5F8C5
:109200000310A878C9B202B0BDE8704004F071BE86
:10921000AB2A00F0E58240F2DA82D5F80310A87894
:10922000C9B202B0BDE8704004F042BEB52A00F0F9
:10923000FB8211D8B12A00F0E582B32A00F0EB825C
:10924000AE2A7FF430AFD5F80310A878C9B202B0C7
:10925000BDE8704004F03DBEB82A00F0F48218D892
:10926000B62A7FF420AFD5F803000028C0F283802F
:10927000AA784C4B03EB82131B7E012B01D005F027
:109280004FF80028CABF484A484A92FBF0F214211E
:1092900078E0B92A00F0E082BA2A7FF404AFD5F86A
:1092A0000300002867DBAA783E4B03EB82131B7E8A
:1092B000012B01D005F034F80028CABF3A4A3B4AD6
:1092C00092FBF0F213215DE0CA2A00F0BA8129D89E
:1092D000C12A00F0978110D8BF2A00F0DB8200F28B
:1092E000E282BC2A7FF4DFAED5F80310A878C9B2B9
:1092F00002B0BDE8704004F0ADBEC32A00F0958115
:10930000C0F08881C92A7FF4CEAE3821A87804F055
:10931000ADFBD5F8033000F4806223F480631A4378
:1093200038212FE0D42A00F0A48111D8D12A00F0EE
:109330009081D22A00F09581CC2A7FF4B4AED5F882
:109340000310A878C9B202B0BDE8704004F02ABE8C
:10935000D62A00F0AC81C0F0A381FB2A00F0BB81CB
:10936000FF2A7FF4A0AED5F80320002A00F0C381C5
:10937000012A00F0CF8104220D4B1A7070E0D5F85D
:1093800003202D21A07803E0D5F803202121A8781F
:1093900002B0BDE8704004F025BB00BFD804002037
:1093A00078F6FF1F780300200024F400B5001000B9
:1093B000F4050020D5F80330A878002BC8BF01229F
:1093C000202104F00FFBAD78AE4BD4F8030001224E
:1093D0005A55AD4B002853F82530B8BF4042984746
:1093E000272102462846D3E7D5F80300AE78A64CDD
:1093F000002854F82630B8BF4042984704EB860650
:109400002021F060A87804F031FB48BBA87804EB79
:1094100080042721E268BBE7AD789C4BD4F80300B9
:1094200000225A55984B03EB85039B699847984B4C
:1094300043F82500A078262153F82020A8E7102122
:10944000A87804F013FB0346DAB2A8780192EA7810
:10945000D2080092C3F307430022102104F070FAEF
:1094600002B070BD3421A87804F000FBD5F80330B9
:109470000246A8781BB942F00202342188E722F0A4
:109480000202FAE73421A87804F0F0FAD5F80330A4
:109490000246A87813B942F00102EEE722F0010279
:1094A000EBE73421A87804F0E1FAD5F803301BB1DA
:1094B00040F01002342165E720F01002FAE7AC78A2
:1094C000714BD5F8030053F8243098472521024604
:1094D00020465DE7AD78D4F8030003EB85039B6974
:1094E0009847282102467DE7AC78D5F8030003EBC6
:1094F00084039B6998472A210246E9E7AC78624BCE
:10950000D5F8030053F8243098472B210246DFE7B3
:10951000D5F803202C2135E7D5F803000028FFF605
:109520002AAFAA785B4B03EB82131B7E012B01D081
:1095300004F0F6FE0028CABF574A584A92FBF0F2E0
:1095400015211FE73421A87804F090FAD5F80330EC
:109550000246A87813B142F008028EE722F0080212
:109560008BE73421A87804F081FAD5F8033002465D
:10957000A87813B142F004027FE722F004027CE7EE
:109580003421A87804F072FAD5F8033013B140F40E
:1095900000628FE720F400628CE7D5F80310A8780A
:1095A000C9B202B0BDE8704004F050BB6E21A8788B
:1095B00004F05CFAEB78AC7801932B7903F00303A9
:1095C00000930022C0F307436E21204646E76E2138
:1095D000A87804F04BFA0246D1B2C2F30722EB7826
:1095E000A878019100926E21002237E7D5F8033068
:1095F000022B3FF6C0AEAA78234B1344EA7883F8D7
:1096000024202DE7AA78234B03EB8213D5F80320FF
:109610001A7225E7AD781C4BD4F8030053F82530B7
:109620009847AD011B4B58511AE7AC78164BD5F84B
:10963000030053F824309847164B03EB841358600B
:109640000EE7A878134BD5F8032003EB80135A8359
:10965000B0E5D5F80310A87802B0BDE8704004F07A
:109660006AB9A8780B4BD5F8032003EB8013DA61B5
:10967000A0E5AA78074B03EB8213D5F803201A6202
:10968000EEE600BF4F03002078F6FF1FD404002051
:10969000C8040020780300200024F400B500100066
:1096A000AA78874B03EB8213EA785A76D8E6D5F886
:1096B000030006F091FF80A3D3E9002307F01CF913
:1096C00041EC100B07F0F0FC51EC100B07F084FAA2
:1096D000112102465BE60021A87804F0C7F9D5F80D
:1096E00003100246A87819B142F0100200214FE69B
:1096F00022F010024CE6A978714B03EB81131A7625
:10970000704B714A43F8212003EB81039A629A61FE
:109710005A63A5E6A9786A4B03EB81131A76694B65
:109720006A4A43F8212003EB8103694A9A62694A35
:109730009A61694AECE7D5F80310A878C9B202B07B
:10974000BDE8704004F028BAD5F80310A878C9B273
:1097500002B0BDE8704004F08BBAA87804F041FB79
:10976000D5F80310AB78C9B228B9184602B0BDE8E5
:10977000704004F0DFBA184602B0BDE8704004F053
:10978000ADBAA87804F02DFBD5F80310AB78C9B2B8
:1097900028B9184602B0BDE8704004F0EBB918468D
:1097A00002B0BDE8704004F0B3BAD5F80310A87851
:1097B000C9B202B0BDE8704004F0C2B9D5F80310D8
:1097C000A878C9B202B0BDE8704004F04DBBD5F82E
:1097D0000310A878C9B202B0BDE8704004F056BBCF
:1097E000D5F80310A878C9B202B0BDE8704004F003
:1097F00029BBD5F80310A878C9B202B0BDE8704003
:1098000004F089BBD5F80310A878C9B202B0BDE84E
:10981000704004F0F7B9D5F80310A878C9B202B0C7
:10982000BDE8704004F088BAD5F803000028FFF6C0
:10983000A2ADAC78234B53F824309847204B03EB70
:10984000841318610CE6D5F80310A878C9B202B0E9
:10985000BDE8704004F01EBAD5F80310A878C9B26C
:1098600002B0BDE8704004F0A9B9D5F80310A8789B
:10987000C9B204F0DFFB0021A87804F0F7F8D5F8AE
:1098800003100246A87811B142F004022EE722F03C
:1098900004027DE5D5F80310A878C9B202B0BDE88E
:1098A000704004F0B5BBD5F80310A878C9B202B077
:1098B000BDE8704004F09ABB2D431CEBE236FA3F42
:1098C0007803002078F6FF1FA1E30000A9E2000062
:1098D00021E30000F1E2000069E3000070B5C64E2C
:1098E000C64C7378A62B354600F0B48200F2A680F1
:1098F000132B00F0E48148D8092B00F0AB8122D86B
:10990000042B00F087810DD8012B00F04481C0F0BA
:109910003F81022B00F04481032B00F0668103237A
:1099200023704EE1062B00F08781C0F07B81072B6E
:1099300000F08A81082BF2D13521B07804F096F836
:10994000C0F340203CE10E2B00F09D810CD80B2B86
:1099500000F08F81C0F082810C2B00F092810D2BE2
:10996000DDD13421B07886E1102B00F09A81C0F06F
:109970009181112B00F09C81122BD0D1B078A04B9B
:1099800003EB80032A215D6B17E11D2B00F0DA81C8
:1099900022D8182B00F0BD8110D8152B00F09D8126
:1099A000C0F09481162B00F09A81172BB7D1B078B4
:1099B000934B03EB800333219D6AFEE01A2B00F0EA
:1099C000B681C0F0AD811B2B00F0B8811C2BA6D155
:1099D000B07804F0FFF9F3E07F2B00F0CC810FD8D2
:1099E0001F2B00F0BE81C0F0B581202B00F0BC81A0
:1099F000212B94D16E21B07804F038F80014DFE008
:109A0000A32B00F01B8208D88C2B00F0BA81A22B6C
:109A100085D1B07804F0BBF9D2E0A42B00F012821B
:109A2000A52B7FF47CAFB07804F0DBF9B378002885
:109A300040F00C82184604F0FCF9C1E0BE2B00F0A7
:109A40006C8245D8B32B00F02E8221D8AB2B00F0CE
:109A50001A820ED8A82B00F00E82C0F00882A92B23
:109A600000F00D82AA2B7FF45AAFB07804F073FA9D
:109A7000A6E0AD2B00F00F82C0F00982AE2B00F003
:109A80000E82B12B7FF44BAFB07804F095F997E0DC
:109A9000B92B00F034820ED8B52B00F02482C0F030
:109AA0001B82B62B00F02982B82B7FF438AFB07838
:109AB00004F09EF984E0BB2B00F02782C0F02382E3
:109AC000BC2B00F02682BD2B7FF429AF712160E012
:109AD000CC2B00F0348228D8C32B00F05E8113D841
:109AE000C02B00F02882C0F02282C12B00F04F81F1
:109AF000C22B7FF414AFB278414B910103EB820388
:109B0000404A9B6A505895E0C52B00F05581C0F043
:109B10004E81C92B00F05381CA2B7FF400AFB2787D
:109B2000384B03EB82135B8BA1E0D22B00F06381F7
:109B300012D8CF2B00F0458104D8CE2B7FF4EFAEA6
:109B40006F2112E1D02B00F05081D12B7FF4E7AED2
:109B5000B07803F0EDFE33E0D62B00F058810BD83F
:109B6000D42B00F04E81D52B7FF4D9AEB278254BA3
:109B700003EB82135B7E7AE0FB2B00F05C81FF2B12
:109B80007FF4CDAEB2781F4B03EB82131B7E6EE0E9
:109B90002D21A87801E02121B07803F067FF0FE0C4
:109BA0002021B07803F062FF154B0128B07803EB59
:109BB00080034FF027019D6A12D103F057FFA84799
:109BC0006060114B1B7853B1104B62681A60104BE8
:109BD000002A40F0B8811A6842F008021A6070BD8D
:109BE00003F044FFA8474042EAE7B078044B03EB98
:109BF000800322219D6AE0E7D8040020F4050020BC
:109C000078F6FF1F78030020EF050020E005002014
:109C1000E0040020B278A84B03EB82039A6AD8686C
:109C20009047CDE7B278A44BA44903EB820351F8E7
:109C300022005B6B9847C3E71021B07803F016FF52
:109C4000C0F30720C000BBE71021B07803F00EFF7F
:109C5000C0B2F7E7B07804F00FFBB1E73521A87880
:109C600003F004FF10F0020F0CBF01230023636018
:109C7000A7E7B078352103F0F9FEC04300F00100FA
:109C80009EE73421EBE7B078342103F0EFFEC0F318
:109C9000001095E7B078884B03EB800324215D6BBF
:109CA0008BE7B078844B03EB800325219D6A84E722
:109CB000B078814B03EB800328215D6B7DE7B078A2
:109CC0007D4B03EB800323219D6A76E7B0787A4BC6
:109CD00003EB80032B219D6A6FE72C215CE71521A4
:109CE000A87803F0C3FE0028D5BF6FF07F43744B04
:109CF000636093FBF0F0AA78724BC8BF606003EB1F
:109D000082131B7E002B7FF45CAF606804F0CCFAFA
:109D100056E73421B07803F0A9FEC0F3C0004FE746
:109D20003421B07803F0A2FEC0F3800048E734216C
:109D3000B07803F09BFEC0F3C02041E7B07804F098
:109D400042F83DE7B0785C4B03EB80039D6A02F07C
:109D50009BFB34E7B078102103F088FEC0F303408A
:109D60002EE71021B078F7E76E21A87803F07EFE89
:109D7000C0F3090024E7B2784F4B134493F8243022
:109D800075E7B07804F011F8C0F1080018E7B27870
:109D90004C4B03EB82131B7A69E7B178494B464A77
:109DA00003EB811302EB81025868926A38E7B278BC
:109DB000454B53F822305AE7B278444BF9E7382143
:109DC000E7E600236360424AB378D15C09B1012120
:109DD00061600021D1543F4AD15C19B1616841F002
:109DE000020161600021D154EBE66F21B07803F0ED
:109DF0003DFE000EE4E6B278324B03EB8213DB69E2
:109E000035E7B2782F4B03EB82131B6A2FE7112142
:109E1000B07803F02BFE06F0DFFB25A3D3E9002387
:109E200006F040FC41EC100B07F0AAF851EC100BC7
:109E300006F0D2FEC4E60021B07826E7B07803F041
:109E4000D0FFBDE6B07803F0DAFFB9E6184603F0BC
:109E5000DDFFB5E6B07803F0C4FFB37818B9184653
:109E600003F08EFFACE6184603F0DCFFA8E6B078FE
:109E700003F074FFA4E6B07804F086F8A0E6B078AA
:109E800004F062F89CE6B07804F057F898E6B078F1
:109E900004F068F894E6B07804F07DF890E6B078C5
:109EA00004F067F88CE6B07803F0C5FF88E600BFE1
:109EB0002D431CEBE236FA3F78F6FF1FC804002062
:109EC0000024F40078030020340300203C04002028
:109ED000700300204C0300206F21B07803F0C6FD12
:109EE000C0F304406CE6B178194B1A4A03EB8113B6
:109EF00002EB81021869926A92E61421F0E6B078CA
:109F000003F04CFF5CE61321EAE6B07804F0CEF8EB
:109F100056E6B07804F0D1F852E60021B07803F0AC
:109F2000A5FD10F004003FF44BAE01239FE6B0788E
:109F300004F0B5F844E6B07804F0AAF840E6B0784A
:109F400004F098F83CE61A6822F0080246E600BFE2
:109F50007803002078F6FF1F38B5BE4A90780228B3
:109F6000144600F0EE80032800F0F280002840F054
:109F7000DC8153784D2B00F0A1803AD8452B79D065
:109F800016D8412B6DD004D8402B63D00322B24B9E
:109F90005EE0422B69D0442BF8D1B049D2F80330AF
:109FA00041F81C3F04221C20BDE83840FEF70DBFDD
:109FB000492B6CD014D8462B61D0472BE6D1A74D46
:109FC000D2F803302946042241F8083F0820FEF762
:109FD000FCFE2A8A29896879BDE8384003F0ACB9CB
:109FE0004B2B60D04C2BD1D19C4BD1789970022057
:109FF00033E0542B00F0838018D8512B6AD008D856
:10A000004F2B60D0502BC1D1944BD178997516202D
:10A0100023E0522B6BD0532BB8D1904DD2F80330A4
:10A020002946042241F8103F1020D0E7842B7ED02F
:10A0300008D8552B6FD0832BA8D1894BD2F8032099
:10A040001A6438BD852B77D0FF2B9FD1D278854BF2
:10A050001A7038BDD17845F2FF70BDE83840FEF780
:10A06000A2BE7E4BD1781970F7E77C4BD17859703E
:10A070000120F2E7794BD17859710520EDE7774956
:10A08000D2F8033041F80C3F04220C208CE7D27840
:10A09000724B1AB9DA75D97D1720DEE76E490122B5
:10A0A000DA754A60F7E76D4CD178E1700320FEF76E
:10A0B0007AFEE078BDE83840FEF754BB674BD178B4
:10A0C00059751520C9E7D2F80310644BC9B2597607
:10A0D0001920C2E7614D2A7DD20704D5E378DB075A
:10A0E00001D4FEF7DDFEE17829751420B5E75B4960
:10A0F000D2F8033041F8203F0422202054E7D2F860
:10A100000330012B00F211815449D37801F81A3F32
:10A1100001221A2048E7D2F80330012B00F2058112
:10A120004E49D37801F81B3F01221B203CE74E4BE0
:10A13000D2F803201A6038BD494BD2F803205A6484
:10A1400038BD5178494BD2F8032043F8212038BD5F
:10A1500053782E2B3FF61AAF01A252F823F000BF1E
:10A160001DA200002FA2000041A200008D9F000050
:10A170008D9F00008D9F00008D9F00008D9F00002F
:10A180008D9F000075A200007FA2000089A2000040
:10A190008D9F00008D9F00008D9F00008D9F00000F
:10A1A0008D9F00008D9F00008D9F00008D9F0000FF
:10A1B0008D9F00008D9F00008D9F00008D9F0000EF
:10A1C0008D9F00008D9F00008D9F000093A20000D6
:10A1D0009FA20000ABA20000B7A20000C3A2000033
:10A1E000CFA200008D9F00008D9F00008D9F00007A
:10A1F0008D9F00008D9F00008D9F0000DBA200005E
:10A20000E5A20000EFA20000F9A2000003A30000F5
:10A210000DA3000017A3000021A30000144BD4F8E5
:10A2200003201A60FEF728FA0D4B986438BD104BD6
:10A23000D4F803205A60FEF71FFA094BD86438BDE2
:10A240000B4BD4F803209A60FEF716FA044B1865FE
:10A2500038BD00BFD8040020F40500200C80FF1F8B
:10A2600078F6FF1FEE050020F00500200006002014
:10A27000480400202E4BD4F80320DA6038BD2C4B64
:10A28000D4F803201A6138BD294BD4F803205A6151
:10A2900038BDD4F80330264ADBB2137638BDD4F883
:10A2A0000330234ADBB2D37638BDD4F80330204ADA
:10A2B000DBB2537638BDD4F803301D4ADBB21377D6
:10A2C00038BDD4F803301A4ADBB2937638BDD4F8DF
:10A2D0000330174ADBB2537738BD154BD4F803204F
:10A2E0001A6238BD124BD4F803205A6238BD104BA5
:10A2F000D4F803209A6238BD0D4BD4F80320DA62FB
:10A3000038BD0B4BD4F803201A6338BD084BD4F882
:10A3100003205A6338BD064BD4F803209A6338BD36
:10A32000034BD4F80320DA6338BD04222FE600BFC4
:10A33000480400202DE9F04FC54EC64F32787A70A0
:10A3400064233B70212AD6F803307B6087B0354602
:10A350003C4601F0EB8000F2C3800E2A00F09085AD
:10A3600039D8072A00F0CB8314D8032A00F04A8298
:10A3700008D8012A00F09B81022A00F0F081022314
:10A380002370E6E1052A00F0B78340F27082FFF700
:10A39000A5FADEE10A2A00F0B88307D8082A00F0FF
:10A3A000B183092AEBD1FFF7D7FDD2E10C2A00F0E7
:10A3B0003A8540F22385B078022800F2CD81737887
:10A3C000012B00F04585C0F04085022B00F043854D
:10A3D00003233B70BDE1182A00F0B3862BD8142A62
:10A3E00000F0078615D80F2A00F06585132AC6D11C
:10A3F0007178994A092900F2D085DFE811F0CB0580
:10A40000D705DA05DD05E105E805EB05EE05F10503
:10A41000E605162A00F0918640F20C868F4AD16D2F
:10A42000072900F29681481C02EB8101D065906DEE
:10A43000086693658DE11C2A00F08A8722D81A2AC3
:10A4400000F0AA8640F28A86844C94F8812072B982
:10A450005E1C04BF804B1B680A205843C4F884006C
:10A46000FEF70AF90123C4F8880084F881306B787C
:10A47000042B00F26E81DFE813F0A006E1060F075F
:10A480003D07B6061F2A00F0988700F2F5871E2ABE
:10A490007FF475AF7278142A00F2BF84B078022876
:10A4A00000F25C8702EB42046D4D044445F8243011
:10A4B0006C4B9B7E002B00F04C81002A00F0498100
:10A4C000032111FB02010C23013A5A4302F5D36325
:10A4D000042205EB810102FB0030FEF776FC38E137
:10A4E000802A01F0FF8044D8402A01F0E38029D877
:10A4F000242A01F079800CD8222A01F06D80232AC9
:10A500007FF43DAF544B1B68C6F80330FFF724FDC2
:10A510001FE1262A01F0A680C1F09980272A7FF446
:10A520002EAFB278022A00F217817378142B00F252
:10A53000748403EB43031344474A1168484A42F8C2
:10A54000231006E1442A01F0C18007D8422A01F015
:10A55000B98041F2B38001F084FFFAE0462A01F0AD
:10A56000BD80C1F0B780472A7FF409AF01F07DFFBD
:10A57000EFE0872A01F05D8146D8832A01F0DE8072
:10A580000AD8812A01F0B480822A7FF4F8AE334BD6
:10A59000022283F85420DCE0852A01F00281314A4E
:10A5A00041F2EC803049314C01250D70B3F5805FEC
:10A5B0009178217081F0FB80127D12EA050641F04E
:10A5C000F680184604A9FEF75DFC9DF81030637014
:10A5D0009DF81130A3709DF81230E3709DF816308D
:10A5E00023719DF8153063719DF81430A3719DF8A7
:10A5F0001330E37126722B46E15C227A01330A4460
:10A60000082B2272F8D1A4E08C2A01F05A813BD8A1
:10A61000892A01F03B81C1F0D4808A2A7FF4AFAE51
:10A620007278134B002A41F049811A70114AEB7875
:10A6300013700A4A92F870110F4A11700F490022E4
:10A640000A700F490A700F4A11780B43137080E0AB
:10A65000D8040020F4050020E005002078F6FF1F54
:10A66000E40400200C80FF1FE4050020E505002025
:10A6700040030020530300209804002052030020D0
:10A68000D704002041030020F22A01F08981FF2A2B
:10A6900001F0CB818D2A7FF472AE7278032A01F229
:10A6A0007B81DFE812F04E09350967097509B37837
:10A6B000022B51D8DFF87882DFF87C92974F002484
:10A6C000AA78E6B2B2420AD0954B03EB8212527ED0
:10A6D000002A3BD003EB84135B7E934236D1E35DCB
:10A6E0004FF0000A04F808A004F809A04FEA840B10
:10A6F00043B18C4B262153F82420304603F072F9E5
:10A7000004F807A0884BD5F803004FF0010A04F8BD
:10A7100003A0864B002853F80B30B8BF404298473F
:10A7200027210246304603F05DF9D5F80330002BAF
:10A73000D8BF02224FF00003D4BF0192CDF804A08D
:10A7400000931A462021304603F0FAF80134032C16
:10A75000B6D107B0BDE8F08F04232370F9E7B378D2
:10A76000022BF9D8DFF8C881DFF8CC916B4F0024B9
:10A77000AA78E6B2B2420AD0694B03EB8212527E4B
:10A78000002A3BD003EB84135B7E934236D1E35D1A
:10A790004FF0000A04F808A004F809A04FEA840B5F
:10A7A00043B1604B262153F82420304603F01AF9B8
:10A7B00004F807A05C4BD5F803004FF0010A04F839
:10A7C00003A05A4B002853F80B30B8BF40429847BB
:10A7D00027210246304603F005F9D5F80330002B57
:10A7E000C8BF02224FF00003CCBF0192CDF804A0F5
:10A7F00000931A462021304603F0A2F80134032CBE
:10A80000B6D1A6E7B378022BA6D8DFF81C81DFF813
:10A810002091DFF824A10026AA78F7B2BA4209D025
:10A820003F4B03EB8212527EEAB103EB86135B7E51
:10A83000934218D1384602F0BDFC012306F80830D7
:10A8400000222721384603F0CDF80024022301938B
:10A850000094234622462021384603F071F806F87A
:10A86000094006F80A400136032ED5D171E7B078C9
:10A87000022803D97278022A7FF46BAF6A78012A22
:10A880005CD005D3022A00F0B9800323237060E76F
:10A89000274FDFF8A480244E0024AA78A24209D0D2
:10A8A0001F4B03EB8212527EA2B303EB84135B7E39
:10A8B00093422FD1A35D4FF0000904F8079004F8EC
:10A8C00008905FFA84FA43B11A4B272153F82420E9
:10A8D000504603F087F804F80690DFF8409014F82B
:10A8E00009304BB10F4B262153F82420504603F07A
:10A8F00079F8002304F80930D5F803202D215046BB
:10A9000003F070F80023019300931A46202150466B
:10A9100003F016F80134032CBFD11AE7D404002049
:10A9200078030020C80400204F03002078F6FF1FA2
:10A930004C03002084F6FF1F70030020DFF8E09234
:10A94000DFF8E0A2DFF8F8B20026AA78B2420AD017
:10A95000AD4B03EB8212527E002A40D003EB8613EC
:10A960005B7E93423BD116F80B300020012B06F89A
:10A97000090006F80A00F7B23AD034D3022B39D0D6
:10A98000A24BF25C804652B1A14A039352F82620B2
:10A990002721384603F026F8039B0022F2549D4BF2
:10A9A000F25C52B19C4A039352F826202621384685
:10A9B00003F018F8039B0022F254D5F803309844B2
:10A9C00042462D21384603F00DF8002301930093F1
:10A9D0001A462021384602F0B3FFC4F8048001363D
:10A9E000032EB2D1B5E62D21384603F03FF8C7E774
:10A9F0002121F9E7384602F09BFFC1E7142B3FF70E
:10AA0000ABAE020642D5DFF81882DFF818927F4F0E
:10AA10000024AB782341DB0734D5E35D4FF0000A17
:10AA200004F808A004F809A0E6B243B1784B272146
:10AA300053F82420304602F0D5FF04F807A0DFF8D1
:10AA4000D4A114F80A304BB1734B262153F82420BB
:10AA5000304602F0C7FF002304F80A30D5F803306F
:10AA60006E4A03EB430323442D2152F82320304642
:10AA700002F0B8FF0023019300931A4620213046CC
:10AA800002F05EFF0134032CC3D162E602283FF6D8
:10AA900063AE634B5D4E00241C54624B1C54335C0C
:10AAA00043B1614B03EB80032721DA6802F09AFF80
:10AAB000AB78F454A878574C235C43B1564B26210D
:10AAC00053F8202002F08EFFAB780022E254D5F834
:10AAD0000330A878514A03EB430303442D2152F875
:10AAE000232002F07FFF0023A878019300931A46E9
:10AAF000202102F025FF2CE6FEF7B8FA29E6FEF742
:10AB0000A7FA26E6FEF7A4FA23E6B378022B00F0B4
:10AB1000D680032B00F0D880002B40F0688173783A
:10AB2000502B00F0A18029D8462B00F08E8010D841
:10AB3000422B66D006D8402B49D0412B5DD0032351
:10AB4000237049E0442B7DD0452BF8D1374B5B79FE
:10AB500055E04B2B7FD009D8472B79D0492BEED12C
:10AB6000324BDB7D003318BF012348E04D2B78D0FA
:10AB700074D34F2BE3D12D4B5B7E40E0802B00F054
:10AB8000828012D8532B75D006D8512B6FD0522B00
:10AB9000D5D1264B1B6A32E0552B71D06DD3562B85
:10ABA000CDD1224B93F8243029E0832B76D006D8E0
:10ABB000812B6CD0822BC2D11B4B9B6D1FE0852B50
:10ABC00072D06ED3FF2BBAD1194B1B78CAE745F26E
:10ABD000FF70FEF721F97860164B1B78002B3FF4CD
:10ABE000B8AD154B62681A60144B002A40F0018121
:10ABF0001A6842F008021A60ABE50C4B1B786360E0
:10AC0000EAE70A4B5B78FAE7780300204F0300205D
:10AC100084F6FF1FD4040020C8040020E4040020B0
:10AC20004C0300207003002078F6FF1F0C80FF1FEC
:10AC3000EE050020EF050020E0050020E0040020E4
:10AC40009CF6FF1FA44BDB69D9E7A34BDB68D6E773
:10AC5000A14B9B68D3E7A04BDB78D0E79E4B9B785A
:10AC6000CDE79D4B5B7DCAE79B4B9B7DC7E79A4B2E
:10AC70001B7DC4E7984B1B69C1E7974B9B7EBEE7E2
:10AC8000954BDB7EBBE7954B93F85430B7E7934B7E
:10AC900093F854301E1F73427341B0E78F4B1B6C07
:10ACA000ADE78F4B1B68AAE78C4A8E48536C43F282
:10ACB000390100FB0313536423F000439FE77278CC
:10ACC000894B53F822309AE773782E2B3FF637AF33
:10ACD00001A252F823F000BF95AD000099AD00002D
:10ACE0009FAD00003FAB00003FAB00003FAB00005A
:10ACF0003FAB00003FAB00003FAB0000D9AB000012
:10AD0000D9AB0000D9AB00003FAB00003FAB000067
:10AD10003FAB00003FAB00003FAB00003FAB00008B
:10AD20003FAB00003FAB00003FAB00003FAB00007B
:10AD30003FAB00003FAB00003FAB00003FAB00006B
:10AD40003FAB0000A3AD0000A9AD0000ADAD000019
:10AD5000B1AD0000B7AD0000BBAD00003FAB0000DF
:10AD60003FAB00003FAB00003FAB00003FAB00003B
:10AD70003FAB0000C1AD0000C5AD0000CBAD000091
:10AD8000D1AD0000D7AD0000DDAD0000E3AD0000A7
:10AD9000E9AD0000554B85E7544B5B682FE7534BFB
:10ADA00057E7524B1B7E2AE7504B6AE74F4BE3E6CF
:10ADB0004E4B1B7F23E74D4B60E74C4B5B7F1EE701
:10ADC0004A4BE7E6494B5B6A19E7484B9B6A16E733
:10ADD000464BDB6A13E7454B1B6B10E7434B5B6B42
:10ADE0000DE7424B9B6B0AE7404BDB6B07E7042305
:10ADF000A6E61A6822F008021A60AAE4B378022BC9
:10AE00000ED17078372808D800F5FF7038498000D7
:10AE100004220144FDF7D9FF9BE40323237098E447
:10AE200004233B7095E4B378022B0BD1707837285C
:10AE3000F3D800F5FF702E49800004220144FDF78D
:10AE4000FDFF86E404233B7083E402F0ABF980E469
:10AE500002F0B0F97DE402F0B5F9264B78601B787A
:10AE6000002B3FF476AC244B1860244B1A6818B9B9
:10AE700042F008021A606CE422F008021A6068E4EA
:10AE8000B278022A14D17078072806D813B9FDF7D2
:10AE9000B7FD5EE4FDF7A0FD5BE4FF287FF459AC4D
:10AEA0005D1C0ABF144BD8B21878FDF7BDFD50E405
:10AEB00004233B704DE4B378012B3ED023B1022B29
:10AEC0005ED004233B7024E07078082818D8FDF782
:10AED000BCFD60601DE000BF0C80FF1F78F6FF1F07
:10AEE000F00500206D4EC6410006002048040020F9
:10AEF00008FEFF1FEF050020E0050020E004002011
:10AF00000A2815D19E4B1B6983F40073C3F34023B9
:10AF10007B609C4B1B78002B3FF41BAC9A4B626808
:10AF20001A609A4B82BB1A6842F008021A6010E459
:10AF3000FF28EED1FDF7C0FDCBE77078092802D0DD
:10AF400002F0CAF9C5E70020FDF7CEFD0546012055
:10AF5000FDF7CAFD06460220FDF7C6FD8642D4BFB6
:10AF6000002301239D4209DD331C18BF01231BB9B7
:10AF700086423546B8BF05466560CAE7031CF4E75C
:10AF80007078FDF77BFDA4E71A6822F008021A60CA
:10AF9000FFF7DFBB10681844106012687B4B12BBD0
:10AFA0001A6842F008021A60FFF7D3BB1068C01A93
:10AFB000F2E710685843EFE7106890FBF3F0EBE717
:10AFC000116891FBF3F003FB10131360E5E71068C1
:10AFD0001840E1E710681843DEE710685840DBE7E7
:10AFE0001368DB43F1E71A6822F008021A60FFF7E2
:10AFF000B0BB654A1168654A8B4213680BDA23F0CF
:10B00000030343F004031360136871B943F00803AA
:10B010001360FFF79EBB0BBF23F0060323F005036D
:10B0200043F0010343F00203EDE723F0080313604C
:10B03000FFF78FBB72780C2A3FF68BABDFE802F08C
:10B04000071019222B343E475059626B74004F4A47
:10B05000126814077FF57DAB4D4A9365FFF779BB06
:10B060004A4A126810073FF574AB494A9365FFF7E7
:10B0700070BB464A1268D1077FF56BAB444A9365B3
:10B08000FFF767BB414A1268D2073FF562AB404AFF
:10B090009365FFF75EBB3D4A126857077FF559ABD2
:10B0A0003B4A9365FFF755BB384A126812F0050F0B
:10B0B0003FF44FAB364A9365FFF74BBB334A1268F8
:10B0C00096077FF546AB324A9365FFF742BB2F4A9E
:10B0D000126895073FF43DAB2D4A9365FFF739BBE6
:10B0E0002A4A1268D4067FF534AB294A9365FFF7E4
:10B0F00030BB264A126890067FF52BAB244A936535
:10B10000FFF727BB214A126851067FF522AB204A80
:10B110009365FFF71EBB1D4A126812067FF519AB37
:10B120001B4A9365FFF715BB184A1268D7057FF5D0
:10B1300010AB174A9365FFF70CBB154A9365FFF7F1
:10B1400008BB134AD36D002B3FF403AB013BD3651F
:10B1500002EB83031B6E9365FFF7FBBA73782E2B0C
:10B1600004D80C4A0121D154FFF7F3BAFF2B7FF426
:10B1700054AE074B012283F88020FFF7EABA00BFE4
:10B1800080F00F40EF050020E0050020E0040020E3
:10B1900078F6FF1F9904002073782E2B04D8B04A4C
:10B1A0000021D154FFF7D5BAFF2B7FF436AEAD4B5B
:10B1B000002283F88020FFF7CCBAFDF75DFAD4F8BF
:10B1C0008830C01A0028D4F88430B8BF4042984272
:10B1D00095BFA36D002303F1FF3384F8813098BF3E
:10B1E000A365FFF7B6BAA87801F0ECFF40B99E4A14
:10B1F00084F88100136823F010031360FFF7A9BAE5
:10B20000D4F88430ABB1FDF737FAD4F88830C01ADF
:10B210000028D4F88430B8BF4042984209D9924AF5
:10B22000002384F88130136843F010031360FFF7A4
:10B2300090BAA36D013BA365FFF78BBAA8783521BF
:10B2400002F014FC10F4007509D0874A002384F83A
:10B250008130136823F010031360FFF77ABAD4F833
:10B260008430A3B1FDF708FAD4F88830C01A00285A
:10B27000D4F88430B8BF4042984208D97A4A84F85A
:10B280008150136843F010031360FFF762BAA36D97
:10B29000013BA365FFF75DBAA878352102F0E6FB14
:10B2A00010F0010509D0704A002384F8813013683A
:10B2B00023F010031360FFF74CBAD4F88430A3B125
:10B2C000FDF7DAF9D4F88830C01A0028D4F88430B1
:10B2D000B8BF4042984208D9634A84F88150136845
:10B2E00043F010031360FFF734BAA36D013BA3656D
:10B2F000FFF72FBAA878352102F0B8FB10F002054D
:10B3000009D0594A002384F88130136823F01003D0
:10B310001360FFF71EBAD4F88430A3B1FDF7ACF97F
:10B32000D4F88830C01A0028D4F88430B8BF40421E
:10B33000984208D94C4A84F88150136843F01003AE
:10B340001360FFF706BAA36D013BA365FFF701BACF
:10B35000444B002283F85420FFF7FBB9FF287FF409
:10B36000FBA9424E3AB300244FF003080C2768783B
:10B3700018FB00410138784300F5D36000EB8400EE
:10B38000042206EB81010134FDF71FFD032CEED1F1
:10B39000FFF7DFB929197819042231440435FDF784
:10B3A00014FD0C2DF6D10C34FC2C3FF4D2A9002551
:10B3B00004F28C67EEE70C24F9E77378142B3FF660
:10B3C0002CADB278022A1BD803EB43031344274A5F
:10B3D00052F82320264B7A601B78002B3FF4B9A942
:10B3E000244B1A60204B2AB91A6842F008021A60EE
:10B3F000FFF7AFB91A6822F008021A60FFF7A9B97F
:10B40000FF2A7FF4A9A9194E3BB300244FF003088B
:10B410000C27687818FB00410138784300F5D360A9
:10B4200000EB8400042206EB81010134FDF706FDE8
:10B43000032CEED1FFF78DB961197819042231443C
:10B440000435FDF7FBFC0C2DF6D10C34FC2C3FF43D
:10B4500080A9002504F28C67EEE70C24F9E700BF11
:10B460009904002078F6FF1FE0040020E404002087
:10B47000EF050020E00500207678142E3FF6CDACD5
:10B48000AF7838062AD5A64FDFF898820024AB782B
:10B490002341D90709D56E782121E0B202F0E6FAFE
:10B4A00006EB4606264447F8260098F81A3083B182
:10B4B0006B7873B1032111FB03410C20013B58430E
:10B4C00000F5D360042207EB810100EB8400FDF757
:10B4D0007CFC0134032CDAD1FFF73BB9022F3FF695
:10B4E0003BA92121384602F0C1FA8E4B8C4C9B7E41
:10B4F00006EB46063E4444F82600002B3FF429A9FB
:10B500006A78002A3FF425A9A878032111FB0201DB
:10B510000C23013A534303F5D363042204EB810166
:10B5200002FB0030FDF751FCFFF713B972787E4B38
:10B530000A2A0CD8DFE802F006151A1F252D32372B
:10B540003C41450079491A6809680A441A601A683A
:10B55000774B002A3AD11A6842F008021A60FFF7C6
:10B56000F8B872491A680968521AEFE76F4A196801
:10B5700012684A43EAE76D491A68096892FBF1F2DA
:10B58000E4E76A4A1868116890FBF1F201FB1202C5
:10B59000DCE766491A6809680A40D7E763491A6810
:10B5A00009680A43D2E761491A6809684A40CDE749
:10B5B0005E490A68D2430A60C9E719685B4A1160AC
:10B5C000C5E75A4A196810681860F8E71A6822F047
:10B5D00008021A60FFF7BDB8534B1B68C6F803306A
:10B5E000FDF744FDFFF7B5B87378052B3FF6B1A81A
:10B5F000DFE803F0030A11181F264D4A136803F011
:10B600000F031360FFF7A5B8494A136823F010032E
:10B610001360FFF79EB8464A136823F020031360B7
:10B62000FFF797B8424A136823F040031360FFF70F
:10B6300090B83F4A136823F080031360FFF789B87E
:10B640003B4A136823F480731360FFF782B8717864
:10B650002E293FF6E2AB374A02EB8102C2F88C306A
:10B66000FFF777B8334B304AD3F8481111602F4AAF
:10B67000D3F84C111160D3F850219A652C4AD3F8B5
:10B6800054111160D3F8582183F88120D3F85C213C
:10B69000C3F88820D3F86021C3F8842093F864119C
:10B6A000254A505C08B101205054002283F86821DB
:10B6B000FFF74FB800F0C0FEFFF74BB800F0BDFE3B
:10B6C000FFF747B800F0CCFEFFF743B800F0CAFE22
:10B6D000FFF73FB800F0C7FEFFF73BB800F0C4FE2D
:10B6E000FFF737B8134B002283F85420FFF731B827
:10B6F00072782AB1012A09D003233B70FFF729B8D9
:10B700000C4B012283F85420FFF723B8B3F5805F78
:10B71000BFF422A8074981F854208B65FFF719B8B8
:10B72000E40400200C80FF1FE0050020FC05002041
:10B73000E004002078F6FF1F99040020C04AC148A9
:10B74000002382F8803082F8683102F18C044FF0D7
:10B75000FF35194644F82350C15401332F2BF9D13A
:10B76000B94B82F854101960B84B91651960B84B09
:10B77000D16582F881101960FEF7EBBF127D920748
:10B780000BD4B3F5805FBEF4E7AFAD4A042182F875
:10B790005410C2F86C31FEF7DCBF08233B70FEF793
:10B7A000D8BFA74B002283F85420FEF7D2BF2B4608
:10B7B0000022E2540133082BFBD123782372FEF7D9
:10B7C000C8BF7378012B19D005D3022B1FD00323D8
:10B7D0003B70FEF7BEBF9F4B01221A709E4B9F4AE3
:10B7E0009B7813709E4B196800230139013311F8BF
:10B7F000010FD054082BF9D1FEF7ABBF0C22FA7120
:10B800007B718E220923BA713B71FEF7A2BF914B67
:10B81000944801221A70904B904A9B781370002331
:10B8200001331918082B11F8091CD154F8D1FEF76F
:10B8300090BF7378032B3EF68CAFDFE803F0021065
:10B840001D227F4B93F85420FA7193F88120D3F88E
:10B850006C31BA711A0A7A713B71FEF77ABF784B74
:10B8600093F85420FA7193F881209B6DBA711A0AEB
:10B870007A713B71FEF76DBF734B1B687B60FEF7FF
:10B8800068BF724B1B687B60FEF763BF7278002A4B
:10B890007EF45FAFB17800297EF45BAF40F2D24214
:10B8A00093427EF456AF45F2FF70FDF77CFAFDF748
:10B8B000F7FA0120FCF7BCFFFEF74BBF0122FEF7B1
:10B8C000B4BE75782DB1012D13D003233B70FEF764
:10B8D00040BF042204A945F2FB70FDF7AFFA049BB8
:10B8E000D6F803209A4206BF01237B607D60FEF7F5
:10B8F00030BFB3782A2B07D104225B4945F2FB7095
:10B90000FDF763FAFEF725BF03233B70FEF721BF67
:10B910004B4CD4F87401002104F5BC7281423EF412
:10B9200018AF52F821509D4201F1010520D102EBE0
:10B930008503043B0138814214D3C4F87401FEF737
:10B9400008BF3F4AD2F8741109299DBF481CC2F8AC
:10B95000740102EB8102092394BFC2F878313B7075
:10B96000FEF7F7BE53F8042F43F8042C0131E2E749
:10B970002946D3E7324A0023C2F87431194602F54A
:10B98000BC7242F8231001330A2BFAD1FEF7E1BE54
:10B990000A237B60FEF7DDBE03233B70FEF7D9BEB2
:10B9A0007378812B7EF4D8AEB378922B7EF4D4AE2C
:10B9B000B379A32B7EF4D0AE7379B42B7EF4CCAEE6
:10B9C0003379C52B7EF4C8AEF378D62B7EF4C4AEA3
:10B9D000FDF725F9FCF750FE0446FCF74DFE001B71
:10B9E0000028B8BF4042B0F57A7FF6DBFCF71EFFB7
:10B9F0001E4B00221A604FF0FF32C3F87021C3F8CB
:10BA00007022C3F87421C3F87422C3F87821C3F8F4
:10BA10007822C3F87C21C3F87C22154B154A1A60A2
:10BA20000120FCF705FFFEF794BE40F2D24293429C
:10BA30007EF48FAE024B012283F8A021FEF789BE6F
:10BA400078F6FF1F99040020E0050020FC05002087
:10BA5000E0040020E40500200C80FF1FE505002025
:10BA60000880FF1F00800000DB04002010E000E0E1
:10BA70000080FF1F785634122DE9F84F424B434E99
:10BA8000DFF844B100241C60414BB4651C60414B9D
:10BA900086F881401C6006F1280906F1180A0BEBB4
:10BAA00084134FEA84081B7E3B4A002B3BD13B4B5F
:10BAB00046F8243049F824304AF82430E7B242F8F6
:10BAC00024302721384601F0D1FF354B43F80800D8
:10BAD000344B0025E5542621384601F0C7FF324B90
:10BAE00043F80800314B3846E554013401F084FE38
:10BAF000032CD4D12E4A2B462946904642F82310D7
:10BB00000133B3F5807FF9D12A4CA37E3BBBE37EA2
:10BB10004BB3637DB3B3FDF747F898B3012386F8C1
:10BB20005430BDE8F88F244B46F82430234B49F8B5
:10BB30002430234B4AF82430224BBFE7791909EB14
:10BB40000700042251440437FDF778F90C2FF5D192
:10BB50000C35FC2DDBD0002705F28C69EEE70C25B7
:10BB6000DFF868A0F7E74FF4FF6540F6D807A5F5C2
:10BB7000FF612846042241440435FDF75FF9BD42C8
:10BB8000F5D1C6E70023CAE7E005002078F6FF1FDD
:10BB9000FC050020E0040020ACF6FF1FA1E300003C
:10BBA00084F6FF1F4F030020C8040020D4040020A7
:10BBB000000600200C80FF1FA9E2000021E3000026
:10BBC000F1E2000069E3000078030020E4040020B3
:10BBD000F7B50F4C07460E4694E803008DE80300C6
:10BBE0000C49C1F803300C4B8A7000220F704E7064
:10BBF0001A70FEF79FFB094A217882F8A1119DE88F
:10BC00000300636884E80300184603B0F0BD00BF7A
:10BC1000F4050020D8040020EF05002078F6FF1F6F
:10BC2000F7B504461F4A63781370A3785370E3781E
:10BC300093702379937163795371A3791A4D1371BA
:10BC4000E379D3700E4695E80300184B00221A7072
:10BC50008DE80300FEF76EFB154B1A786F462B46F6
:10BC60009AB9327072702A78B2706A78F270EA7992
:10BC70003271AA7972716A79B2712A79F27197E890
:10BC8000030083E8030003B0F0BD012AF7D109489F
:10BC9000721EF11D10F8014F02F8014F8A42F9D1CE
:10BCA000EDE700BFD8040020F4050020EF050020D8
:10BCB000E4050020E5050020014B93F8A101704741
:10BCC00078F6FF1F2DE9F043994B9A4C1B788FB003
:10BCD0006BB1994B1B78063BDBB2192B04D8974A02
:10BCE00022FA03F3D90702D4002384F8703194F8C0
:10BCF0007031934E5A1E012A51D89249012BCA68BD
:10BD0000079214BF082307238DF81830327894F86F
:10BD1000A2318DF8193000238DF81A30002A33D162
:10BD20008B688DF82030884B8DF8272019788DF896
:10BD3000211059788DF82210D9798DF8231099792E
:10BD40008DF8241059791B798DF825108DF826303F
:10BD500006A801F0DFFB002800F01F837B4B1A7858
:10BD60009846002A00F01E81794B7A4F1B78013BE0
:10BD7000062B00F21381DFE813F0F100F100580107
:10BD80001101110111017F01012AE1D17248013332
:10BD900006AA1A44195CD171082BF8D1D8E7032BF5
:10BDA0003DD1337883BBDFF89C81674F98F8020060
:10BDB00098F801503B7805441D447B781D44FB797D
:10BDC0001D44BB791D447B791D443B791D44FCF720
:10BDD0008DFC98F80100FCF789FC3878FCF786FCAC
:10BDE0007878FCF783FCF879FCF780FCB879FCF7ED
:10BDF0007DFC7879FCF77AFC3879EDB2FCF776FCBB
:10BE00002846FCF773FCA9E7012BA7D1524F002568
:10BE1000785D0135FCF76AFC092DF9D19EE7042B0A
:10BE20002BD1484FDFF82081B8787D78002301229C
:10BE30000544154488F8013088F80020C8F804301B
:10BE4000FCF754FC7878FCF751FC98F80000FCF7FC
:10BE50004DFC98F80100FCF749FC98F80700FCF746
:10BE600045FC98F80600FCF741FC98F80500FCF743
:10BE70003DFCEDB298F80400C0E7072B37D13378CA
:10BE800053BB304B9F7893F801802F4B8DF8007097
:10BE90001D785878D9798DF8025047443D449A79F5
:10BEA0008DF80300284493F805C08DF80410014470
:10BEB00093F804E08DF805200A440CEB0203734468
:10BEC0008DF801808DF806C08DF807E08DF80830F8
:10BED0006846FCF7A1FE41E7012BF9D11E4900237A
:10BEE0005A5C0DF803200133092BF9D1F0E7082B38
:10BEF0007FF434AF144A13490023012053701070AB
:10BF000053608A7849788DF800200A4402448DF8FD
:10BF100001108DF802008DF803308DF804308DF893
:10BF200005308DF806308DF807308DF80820CFE702
:10BF3000EE05002078F6FF1FD80400201102000251
:10BF4000E40500200C80FF1FF4050020D70400202A
:10BF50009804002052030020E5050020AE4A3978FD
:10BF600093688DF8303080238DF831308A238DF836
:10BF7000323000238DF833308DF834308DF8353081
:10BF80008DF836108DF8293007218DF82A300AA84F
:10BF9000D3688DF828100B9301F0BCFA00233B7096
:10BFA00088F80030002384F87031337094F8A031A1
:10BFB00013B10120FCF73CFC06A801F037FA064655
:10BFC000002800F04181954B9DF820201A709DF8C3
:10BFD00021205A709DF822209A709DF823209A7192
:10BFE0009DF824205A719DF825201A719DF826206D
:10BFF000DA709DF8193084F8A231FCF73DFB884BCC
:10C000001860884B00221A709DF81830072B0CBF5F
:10C010000123022384F8703194F854305A1E012A07
:10C020004AD9052B48D0012247E0DFF8EC913B7854
:10C0300099F8020099F8015005440A351D44FCF7AF
:10C0400055FB99F80100FCF751FB8020FCF74EFBF3
:10C050008A20FCF74BFB0020FCF748FB0020FCF794
:10C0600045FB0020FCF742FBEDB23878FCF73EFBC5
:10C070002846FCF73BFB91E7674A507893788DF8A8
:10C080000C303A788DF80D00802103448DF80E10A5
:10C090000A338A218DF80F101344002103A88DF86C
:10C0A00010108DF811108DF812108DF813208DF8E6
:10C0B0001430FCF7B1FD71E700225B4B1A7094F865
:10C0C0005430042B04D1554B19780A0640F168818D
:10C0D00094F87021082A04D840F25113D340DF07A6
:10C0E00001D4FEF727F994F87031092B6FD1FCF7D2
:10C0F000C3FAA36C4D4DC01A00282A68B8BF40424D
:10C10000904208D94A4B1A78012A04BF02221A70B9
:10C11000FCF7B2FAA064FCF7AFFAE36C6A68C01AE5
:10C120000028B8BF4042904208D9414B5A78012AB2
:10C1300004BF02225A70FCF79FFAE064FCF79CFAF5
:10C14000236DAA68C01A0028B8BF4042904208D99F
:10C15000374B9A78012A04BF02229A70FCF78CFAB6
:10C16000206594F8803093B394F868317BBB304AF3
:10C1700030481D46D15C022940F0068150F823105A
:10C180004E1C00F000812C4A84F864311268C4F817
:10C1900048212A4A1268C4F84C21A26DC4F85021E3
:10C1A000274AA1651268C4F8542194F88120C4F884
:10C1B00058210023D4F88820C4F85C2184F8813009
:10C1C000D4F88420C4F86021012384F8683194F8FD
:10C1D0007031092B06D194F85420022A04BF05229D
:10C1E00084F85420D4F87421002A00F0D680092B5A
:10C1F00040F0D38094F85430012B40F0CE80A16DF4
:10C200001048002350F823508D4240F0C28005238F
:10C2100084F85430C1E000BF0C80FF1FD804002018
:10C220008804002030030020EF050020480400208F
:10C230009904002004F7FF1FE0050020FC05002002
:10C24000E0040020F0F7FF1F03A8FCF767FA05469B
:10C2500000284ED0FCF77AFA08B184F8A36194F86C
:10C26000A3219DF80C10531CDBB22244092B84F847
:10C27000A33182F8A4117FF422AF5E4A94F8A4118E
:10C2800052780023914284F8A3317FF418AF5A49C1
:10C290005A5C01331644082BF6B2F9D194F8AC314C
:10C2A000B34222D1554B94F8A5211A7094F8A621D7
:10C2B0005A7094F8A7219A7094F8A8219A7194F86A
:10C2C000A9215A7194F8AA211A7194F8AB21DA7055
:10C2D000FCF7D2F94A4B4B4A186000231370032233
:10C2E00084F8702184F8A33196E6042384F8703131
:10C2F000E5E60AAE3046FCF77CFC48B32B46F25C20
:10C3000001331544082BEDB2F9D19DF83020AA4233
:10C31000ECD13A4B9DF829201A709DF82A205A70CA
:10C320009DF82B209A709DF82C209A719DF82D2055
:10C330005A719DF82E201A719DF82F20DA70FCF7A3
:10C340009BF92F4B18602F4B00221A70072361E6D0
:10C3500094F85430013B012B3FF6B1AEA36DB3F519
:10C36000805F0CD2FCF720FC48B1A06D2349431C30
:10C37000A365FCF787FD092384F8703153E6002399
:10C3800084F854309BE6D55401332F2B7FF4F2AE62
:10C390001DE701339A427FF435AF0FB0BDE8F0835B
:10C3A00094F87001082804D840F25112C240D20714
:10C3B000F3D4D4F86C01144DD3F803306970B0F5A0
:10C3C000805F6B6012D20D49FCF748FD0B49D4F831
:10C3D0006C01FCF799FD38B1D4F86C310133C4F825
:10C3E0006C3165232B70D8E70723FBE707232B70FD
:10C3F00000230DE70C80FF1F1CF8FF1FD80400204E
:10C400009004002097040020F4050020704710B528
:10C41000074CFCF731F92368C01AB0F5FA7F05D94B
:10C42000044B0222DA60FCF727F9206010BD00BF40
:10C43000000A002000F00F407047064B5A7832B9CE
:10C44000D3F80310044B01B901221A70704703227C
:10C45000024BFAE7D80400204B030020F40500202B
:10C460007047704770477047704708B5034B3B21D2
:10C47000987801F0FBFA024B586008BDD804002000
:10C48000F405002000000000014B53F82000704725
:10C4900028F8FF1F2DE9F74FB14CE369C3B1B14D47
:10C4A0002E78AEB9FCF7E8F8AF4B1B68C01A00282D
:10C4B000E369B8BF404298420AD9304601F0BCFE59
:10C4C000012001F0B9FE022001F0B6FE01232B701D
:10C4D000236AC3B1A54D2E78AEB9FCF7CDF8A44BB5
:10C4E0001B68C01A0028236AB8BF404298420AD984
:10C4F000304601F0A1FE012001F09EFE022001F075
:10C500009BFE01232B709B4CFCF7B6F8237E04EBBB
:10C510008303DB68C01A0028B8BF40420A2828DD20
:10C52000FCF7AAF821210746207E01F09FFA94F833
:10C53000188004EB88050646EB69C31A07EE903AAB
:10C54000EB68FB1AB8EEE77A07EE903AF8EEE77A76
:10C55000C7EE276A16EE900A04F050F87EA3D3E9DE
:10C56000002304F09FF804F037FB44F82800EF6044
:10C57000EE613521207E01F079FA10F04009054680
:10C580000DD0207E01F058FE237E7B4A0121D1543C
:10C590000F337A4AD15C012904BF0221D154207E95
:10C5A000774E06EB80131B69002B55D0222101F03A
:10C5B0005DFA277E06EB871300281B69B8BF40424F
:10C5C000984249D9E31993F8283073B93421384691
:10C5D00001F04CFA342140F48062384601F002FA4E
:10C5E000237E0122234483F8282094F82B70DFF85F
:10C5F00098B157B9F8B2FCF728FA0BF807000137E1
:10C60000082FF7D1012384F82B305E49DFF86CA1A5
:10C6100027274FF0000802225FFA88F08DE8060015
:10C62000FCF713FA1BF8083083429DE806002ED071
:10C6300008F108030BF8080051F82330022B1FD033
:10C64000032B02D0012B22D108B31AF80730012B9B
:10C6500008BF0AF807201AE0277EE31993F828306C
:10C66000002BC2D03421384601F000FA342120F4E6
:10C670008062384601F0B6F9237E00222344B2E7F7
:10C6800028B91AF80700012801D10AF8073008F183
:10C690000108B8F1080F07F10107BDD1237E15F09D
:10C6A000010104EB03023ED092F8341089B9012154
:10C6B00082F83410334A1A44127E12F0010F08D067
:10C6C00002211B2211FB03232C4AD05C012808BF46
:10C6D000D154237E15F0020104EB03022FD092F80F
:10C6E000371089B9012182F83710264A1A44D27EC0
:10C6F00012F0010F08D00E33204A12F8131001294E
:10C7000004BF022102F8131015F080013ED0237EF1
:10C710001A4A0333D05C012801D10220D054B9F168
:10C72000000F3FD035E092F834000028D1D082F8D5
:10C730003410144A1A44127E12F0020FBFE792F826
:10C7400037000028E0D082F837100E4A1A44D27E13
:10C7500012F0020FCEE700BFFCA9F1D24D6290406B
:10C760000C80FF1F9704002090040020300300205D
:10C770008804002028F8FF1F70030020990400207F
:10C78000780300204804002054F8FF1FB9F1000F7F
:10C790001CD0237E2A4A0F33D05C012804BF02201C
:10C7A000D05499B12749237E0A7842FA03F0C00792
:10C7B0000CD50120244F00FA03F33B70234F38704F
:10C7C0002348007810B922EA03030B70207EC022B0
:10C7D000352101F007F9207E06EB80131B6A0BB3AD
:10C7E0006B051FD4392101F041F921210546207E36
:10C7F00001F03CF9237E06EB8316281A0028326AE2
:10C80000B8BF404290420DD9184601F015FD237E75
:10C81000104A0121D1541533094AD15C012904BFC2
:10C820000221D154207E00F045F8237E0133DBB293
:10C83000022B88BF0023237603B0BDE8F08F00BF32
:10C84000990400205303002052030020D704002045
:10C85000400300204C03002073B5134E335C0446A4
:10C860000D463BB1114B262153F8202001F0BAF8B8
:10C870000023335585EAE572A2EBE57220462721B5
:10C8800001F0B0F80A4B0122002D1A554FF00003B9
:10C89000D8BF0222019200931A462021204601F0BF
:10C8A0004FF802B070BD00BFD4040020C8040020BF
:10C8B0004F0300202DE9F04F0446974EA50177194C
:10C8C000352187B001F0D2F8397A7F6811F0400F36
:10C8D00002464FEA500300F0010024D003F00109A2
:10C8E000C3B27059C0F1000A784203900F0601F0FC
:10C8F0003F080592049320461DD501F0BDFC049B22
:10C90000059AB0FA80FB4FEA5B1B08F1FF3107295B
:10C9100078D8DFE811F01A001A001A001A0058023D
:10C920005802580258025FFA80F903F0010356F8E2
:10C9300005A00397DAE701F09FFC10F1000B18BF88
:10C940004FF0010B059A049BDFE7744F395D013905
:10C950000E2957D8DFE811F00F00350059006500A7
:10C960008800A300C400EA004301A601AC01560000
:10C97000FF011B020402DFF8ACA1DFF8ACB14FF0FD
:10C9800000095FFA89F0844207D073195B7E63B1B6
:10C9900006EB8912527E9A4207D1342101F066F8E3
:10C9A00001234AF8290009F80B3009F10109B9F10E
:10C9B000030FE6D1A8F10208B8F1010F2ED8022327
:10C9C0002DE007EB840334215A68204642F002022E
:10C9D00001F008F84FF0000835445FFA88F084420F
:10C9E00006D06B7E3BB106EB8812527E9A4202D192
:10C9F0005146FFF731FF08F10108B8F1030FECD100
:10CA000007F8048007B0BDE8F08F002BFAD0212191
:10CA1000204601F02BF8424B43F8240004233B55F9
:10CA2000F0E707EB840334215A68204642F0010204
:10CA300000F0D8FF4FF00008CAF1000A35445FFA51
:10CA400088F0844206D06B7E3BB106EB8812527EA2
:10CA50009A4202D15146FFF7FFFE08F10108B8F1F2
:10CA6000030FECD10523DAE7B9F1000FCAD04FF07C
:10CA7000000835445FFA88F39C4206D06B7E3BB1D8
:10CA800006EB8812527E9A4202D1404601F0D4FB56
:10CA900008F10108B8F1030FECD10623BFE707EB5B
:10CAA000840334215A68204622F0030200F09AFFE2
:10CAB0004FF0000835445FFA88F0844206D06B7E60
:10CAC0003BB106EB8812527E9A4202D10399FFF7DE
:10CAD000C3FE08F10108B8F1030FECD107239EE76C
:10CAE000B9F1000F8ED1039B3544C3F100085FFA02
:10CAF00089F0844206D06B7E3BB106EB8912527EF0
:10CB00009A4202D14146FFF7A7FE09F10109B9F1A6
:10CB1000030FECD1082382E77803002064F8FF1F9D
:10CB20003403002068F8FF1F4F030020B9F1000F05
:10CB30003FF468AF2121204600F098FF4FF0000835
:10CB4000824606EB05095FFA88F0844207D099F81F
:10CB500019303BB106EB8812527E9A4202D1002175
:10CB6000FFF77AFE08F10108B8F1030FEBD1BC4AD8
:10CB7000DFF8FCB252F82430A3EB0A0342F8243069
:10CB80004FF000085FFA88F94C4507D073195B7EB7
:10CB9000F3B106EB8812527E9A4219D15BF8282035
:10CBA000342122F00302484600F01CFF039A27219B
:10CBB000484600F017FF52462D21484600F012FF6C
:10CBC0000023019300931A462021484600F0B8FE46
:10CBD00008F10108B8F1030FD4D109231FE791052B
:10CBE0007FF510AF2121204600F040FF9D4B4FF014
:10CBF0000009186006EB050A5FFA89F0844207D045
:10CC00009AF819303BB106EB8912527E9A4202D152
:10CC10000021FFF721FE09F10109B9F1030FEBD162
:10CC20004FF000095FFA89FA544507D073195B7E0B
:10CC30009BB106EB8912527E9A420ED100222D2121
:10CC4000504600F0CFFE00222121504600F0CAFEDF
:10CC500000223921504600F0C5FE09F10109B9F161
:10CC6000030FDFD1A8F10308B8F1010F76D8039BB9
:10CC70004FF00008C3F1000935445FFA88F08442A0
:10CC800006D06B7E3BB106EB8812527E9A4202D1EF
:10CC90004946FFF7E1FD08F10108B8F1030FECD1B7
:10CCA0000A23BCE6B9F1000F3FF4ACAE0B23B6E6A5
:10CCB000B9F1000F7FF4A6AE2121204600F0D6FE88
:10CCC00006EB050883465FFA89F0844207D098F89E
:10CCD00019303BB106EB8912527E9A4202D10021F3
:10CCE000FFF7BAFD09F10109B9F1030FEBD1DFF844
:10CCF00080A14FF0000802239BFBF3FB5FFA88F949
:10CD00004C4507D073195B7EF3B106EB8812527E57
:10CD10009A4219D15AF82820342122F003024846B9
:10CD200000F060FE039A2721484600F05BFE5A4659
:10CD30002D21484600F056FE0023019300931A4629
:10CD40002021484600F0FCFD08F10108B8F1030F6E
:10CD5000D4D10D2363E692057FF554AE0E235EE633
:10CD60004FF0000835445FFA88F0844206D06B7EAD
:10CD70003BB106EB8812527E9A4202D10021FFF7A6
:10CD80006BFD08F10108B8F1030FECD1E6E7DFF81D
:10CD9000E0904FF0000835445FFA88F0844206D0F6
:10CDA0006B7E4BB106EB8812527E9A4204D159F841
:10CDB0002820342100F016FE08F10108B8F1030F15
:10CDC000EAD100232BE6284F395D01390E293FF6C1
:10CDD00019AE01A050F821F015CE000075CE00006C
:10CDE000D1CE0000F3CE000053CF000005CA0000F2
:10CDF00073CF000005CA000005CA000025D000005E
:10CE00003DD00000C9CF0000BBD0000067D10000BA
:10CE100039D10000154BDFF858A001221A554FF008
:10CE2000000935445FFA89F0844206D06B7E4BB12D
:10CE300006EB8912527E9A4204D1342100F016FE8C
:10CE40004AF8290009F10109B9F1030FEAD1B8F153
:10CE5000060F3FF4B4ADB8F1080F7FF4DFADAEE5D7
:10CE6000340300203C04002064F8FF1F4F0300201F
:10CE700068F8FF1FB8F1060F21D107EB84035A6849
:10CE800022F0030242F002023421204600F0AAFD03
:10CE90004FF0000835445FFA88F0844206D06B7E7C
:10CEA0003BB106EB8812527E9A4202D15146FFF7FF
:10CEB000D3FC08F10108B8F1030FECD1A0E5B8F1FB
:10CEC000080FE5D107EB84035A6822F00302DBE781
:10CED000A8F10502012A06D82BB1B8F1060F3FF4DC
:10CEE0009DAD0F239BE5BBF1000F3FF48BAD0C23F1
:10CEF00095E5B8F1050F23D107EB84035A6822F0BA
:10CF0000030242F001023421204600F06BFD4FF095
:10CF10000008CAF1000A35445FFA88F0844206D05E
:10CF20006B7E3BB106EB8812527E9A4202D151468B
:10CF3000FFF792FC08F10108B8F1030FECD191E57D
:10CF4000B8F1070FE3D107EB84035A6822F003021C
:10CF5000D9E7A8F10503012B06D8B9F1000F03D0DA
:10CF6000B8F1050FBDD12AE5BBF1000F3FF44AAD82
:10CF7000B4E5BBF1000F7FF445ADA8F10708B8F1A7
:10CF8000010F0AD907EB840334215A6822F0030207
:10CF900042F00202204600F025FD4FF00008354423
:10CFA0005FFA88F0844206D06B7E3BB106EB8812B4
:10CFB000527E9A4202D10399FFF74EFC08F1010814
:10CFC000B8F1030FECD16BE6BBF1000F7FF41AADA3
:10CFD000A8F10708B8F1010F0AD907EB840334213F
:10CFE0005A6822F0030242F00102204600F0FAFCE7
:10CFF000039B4FF00008C3F1000935445FFA88F045
:10D00000844206D06B7E3BB106EB8812527E9A4278
:10D0100002D14946FFF720FC08F10108B8F1030FDF
:10D02000ECD13DE6BBF1000F3FF4ECAC21212046F2
:10D0300000F01CFD07EB8403186137E6BBF1000F1D
:10D040007FF4E0AC2121204600F010FDDFF850A174
:10D05000049007EB84095FFA8BF8444507D07319F5
:10D060005B7E23B306EB8B12527E9A421FD15AF895
:10D070002B20342122F00302404600F0B3FC039A37
:10D080002721404600F0AEFC049BD9F810202D214A
:10D090001A444046022392FBF3F200F0A3FC002363
:10D0A000019300931A462021404600F049FC0BF101
:10D0B000010BBBF1030FCED14BE693057FF5A2AC7C
:10D0C0000E23212120463B5500F0D0FC334B002796
:10D0D000186006EB0508F8B2844207D098F81930BA
:10D0E0003BB106EB8712527E9A4202D10021FFF734
:10D0F000B3FB0137032FEED100275FFA87F84445D1
:10D1000007D073195B7E9BB106EB8712527E9A4261
:10D110000ED100222D21404600F064FC0022212186
:10D12000404600F05FFC00223921404600F05AFCE6
:10D130000137032FE1D165E44FF0000835445FFA71
:10D1400088F0844206D06B7E3BB106EB8812527E9B
:10D150009A4202D10021FFF77FFB08F10108B8F1E4
:10D16000030FECD1FAE5DFF838904FF000083544B2
:10D170005FFA88F0844206D06B7E4BB106EB8812D2
:10D18000527E9A4204D159F82820342100F02AFC1A
:10D1900008F10108B8F1030FEAD112E63C040020BF
:10D1A00068F8FF1F024B1A5C0AB901221A54704733
:10D1B00064F8FF1F024B1A5C0AB10F221A54704721
:10D1C00064F8FF1F014B185C704700BF64F8FF1F35
:10D1D0000C4A116940F273234B434FF6FF71B3FBC6
:10D1E000F1F36E2B06D9084B4FF480215960572379
:10D1F000136070474F2B9EBF034B4FF48021996003
:10D20000F5E700BF00B0034080F00F401B4B1A68E9
:10D2100002F01F02072A2ED8DFE802F0040B2D11BE
:10D22000171D23291A69164992B20A8041221A60F1
:10D2300070471A69124992B24A804322F7E71A6985
:10D240000F4992B2CA804422F1E71A690C4992B29E
:10D250000A814522EBE71A69094992B24A814622BE
:10D26000E5E71A69064992B28A814722DFE71A691F
:10D27000034992B2CA814022D9E700BF00B00B40F7
:10D2800080F8FF1F38B541F23001114B5A5842F077
:10D2900000625A5041F23C0100245A5842F00062A8
:10D2A0005A5003F5E8230C2540229D604920DC609C
:10D2B0005C621A6001F094F8064B57229D602720AB
:10D2C000DC605C621A60BDE8384001F089B800BFDC
:10D2D0000070044000B003400B2829D8DFE800F0BC
:10D2E000060A0D102828282813281E23114B1889F8
:10D2F00080B270470F4B5889FAE70E4B9889F7E7D1
:10D300000C4BD889F4E70B4B588883B240F273205A
:10D3100058434FF6FF7390FBF3F07047054BD888E6
:10D3200083B28E20F4E7034B188883B24220EFE7E4
:10D330000020704780F8FF1F30B52E4D41F23C04AD
:10D340002B5943F010032B512B4B4FF400741C63EB
:10D350006FF4F8755C63A3F51433A4F13E542C44C8
:10D360001C604FF400545C60244C1C601C68E40199
:10D37000FCD50138072834D8DFE800F0312F2D2BF9
:10D38000293327041E4858601E4B002058631E484E
:10D3900018601E484FF0806400EA8145C3F8804061
:10D3A000C3F88450FAB100EA8240C3F89040C3F851
:10D3B00094004FF08460C3F8A000C3F8A410AAB191
:10D3C000C3F8B000C3F8B42030BD1148DBE7114802
:10D3D000D9E71148D7E71148D5E71148D3E71148F5
:10D3E000D1E71148CFE7C3F89020E2E7C3F8B020B7
:10D3F00030BD00BF00700440009004400F0080501A
:10D400008720FE01004002400F0080000000FC1F4A
:10D410008720FE038720FE0F8720FE138720FE272C
:10D420008720FE638720FEC78720FE07384AD2F890
:10D430008030C3F30363022B5FD0D2F89030C3F384
:10D440000363022B5BD0D2F8A030C3F30363022B3B
:10D4500006D0D2F8B030C3F30363022B56D10323B6
:10D460001B0103F1402202F50032D2F88010C1F313
:10D4700003410170D2F8801011F4801118BF01210E
:10D480008170D2F8801011F4001118BF0121417091
:10D490004178B1BBD2F88410C1F38A4103F1402333
:10D4A00003F500334160D3F88810090E0172D3F8F8
:10D4B0008810090C4172D3F88810090A8172D3F8D8
:10D4C0008810C172D3F88C10090E0173D3F88C1038
:10D4D000090C4173D3F88C10090A8173D3F88C308E
:10D4E000C373D2F880309B024CBF4FF084634FF07F
:10D4F0008063C2F88030012070470023B0E7012329
:10D50000AEE7D2F8841021F06041C7E700207047F1
:10D5100000400240184AD2F87031C3F303630C2B69
:10D5200010B527D04478436804B3C3F31103C2F89D
:10D5300074318368104A1BBAC2F87831C3681BBAC9
:10D54000C2F87C318378002C14BF4FF042624FF058
:10D5500040620BB142F4801203781B0403F4702381
:10D560001343054A0120C2F8703110BD034901EA96
:10D570008343DCE7002010BD004002400000FC1F98
:10D580000B4B4FF00062C3F870214FF48022C3F8B8
:10D590007421084AC3F878216FF48471A2F16632CD
:10D5A0000A44C3F87C21044AC3F87021704700BFC5
:10D5B00000400240785634120000080C10B53A4B77
:10D5C000DA7842F00202DA70384A1078C0B20228E3
:10D5D000114641D0032835D0012832D154689168D2
:10D5E0008C4215D2D978C90707D45168D0684C1C31
:10D5F0005460425CD2B21A7110BD997801F0DF011B
:10D600009970997801F0EF0199701074002317E078
:10D61000517C01F0FF0049B9997801F0DF01997060
:10D62000997801F0EF019970107010BD997841F070
:10D6300004019970917CC9B21971002353740323BA
:10D64000137010BD997801F0EF0199701B79516941
:10D65000DBB20B700223F3E79469D06984421DD2D8
:10D66000D2698869121A012A05D19A7802F0DF027C
:10D670009A7000230B70CB698A699B1A022B9FBF9B
:10D68000094A937843F0080393708A694869531CE8
:10D690008B61054B1B79DBB2835410BD997801F087
:10D6A000DF019970B2E700BF0070064094F8FF1FD9
:10D6B00041F234020A498B5843F080038B50094BE6
:10D6C0004FF418729A62DA6203F5E0331B225A7043
:10D6D000C0229A7000225A71192000F081BE00BF4A
:10D6E0000070044000B0044010B5104B00241C74BE
:10D6F0005C749A6001225C601A700D4AD96091785E
:10D7000001F0F7019170917841F0100191709178DA
:10D7100000F0FE0041F02001917010711A78002A8B
:10D72000FCD1187CB0FA80F0400910BD94F8FF1FBE
:10D730000070064010B5104B00241C745C74DA6154
:10D7400003229C611A700D4A5961917801F0F7012A
:10D750009170917841F010019170917840F0010042
:10D7600041F02001917010711A78002AFCD1187CC8
:10D77000B0FA80F0400910BD94F8FF1F0070064019
:10D7800070B5144C002563610126049B25746674F2
:10D79000A2606560E36140EA0603A561A3740E4BD5
:10D7A000E16026709A7802F0F7029A709A7842F057
:10D7B00010029A709A7800F0FE0042F020029A70EF
:10D7C00018712378002BFCD1207CB0FA80F040093E
:10D7D00070BD00BF94F8FF1F0070064000000000FD
:10D7E00010B50024E0B24FF480323A21013400F049
:10D7F000F9F8032CF6D110BD2DE9F7434A4D05EB9E
:10D8000080150446EB690BB16E8B96B93821204622
:10D8100000F02CF9382120F48062204600F0E2F874
:10D820004FF480323A21204603B0BDE8F04300F0C7
:10D83000D9B800F0BAFAC0F1080006FA00F002F018
:10D84000CBFEED69064685EAE570A0EBE5700F4674
:10D8500002F0C2FE02460B463046394603F04CF851
:10D860000022324B8046894602F01CFF0F460646D6
:10D8700047EC106B684603F09BFA0022002351EC42
:10D88000100B03F077F9A0B13046394603F0A4F944
:10D89000002D06464FF03801B8BF4642204600F042
:10D8A000E5F8382120F48062204600F09BF83246EB
:10D8B000B8E7684649EC108B03F07AFA002D57EC74
:10D8C000106BDDE9000118DD03F086F914A3D3E93C
:10D8D000002305043946304602F0E4FE03F07CF9EB
:10D8E00005433821204600F0C1F8382140F4806219
:10D8F000204600F077F82A4694E703F06DF908A374
:10D90000D3E90023C5433946304602F0CBFE03F08D
:10D9100063F9C0F51C502D041030E1E7AFF300802F
:10D92000000000000088C340780300200000F040A1
:10D93000392100F09BB80A46392100F053B800BFE6
:10D940002DE9F74F01F07F05352D1C46074693461C
:10D950009DF830909DF83480204E4FEA022314D178
:10D960001C4349EA042448EA04249F3024F47364E5
:10D9700024F00304E40456F82030E40C23EA040401
:10D9800046F8204003B0BDE8F08F154A019332F805
:10D9900010A041F0800100225046FBF795F90022CB
:10D9A00059465046FBF790F9214600225046FBF7B6
:10D9B0008BF9002249465046FBF786F90122414681
:10D9C0005046FBF781F9019B1C4349EA042405EB0F
:10D9D0004500384448EA0424D2E700BFB4F8FF1FEA
:10D9E000381201002DE9F04101F07F05352D064682
:10D9F0001446DFF874800FD100F19F0522F47364A0
:10DA000024F0030458F82530E404E40C23EA04036A
:10DA100048F82530BDE8F081124B33F81070002231
:10DA200041F080013846FBF74FF90022210E3846BD
:10DA3000FBF74AF905EB45050022C4F307413846D8
:10DA4000FBF742F935440022C4F307213846FBF7BF
:10DA50003BF90122E1B23846FBF736F948F8254098
:10DA6000BDE8F08138120100B4F8FF1FF8B5324B61
:10DA700001F07F055A190646127B002A54D033F86C
:10DA80001070002229463846FBF71EF90022114685
:10DA90003846FBF719F9002211463846FBF714F90E
:10DAA000002211463846FBF70FF9012200213846C3
:10DAB000FBF70AF9002211463846FBF705F9002268
:10DAC00011463846FBF700F9002211460402384699
:10DAD000FBF7FAF80022114604433846FBF7F4F846
:10DAE00024020443012200213846FBF7EDF824020A
:10DAF000352D40EA04000ED1104A06F19F0552F878
:10DB0000253023F4736323F00303DB04DB0C184399
:10DB100042F82500F8BD222D01D0422D0AD1030282
:10DB200008D540F07F40F8BD05EB45050544034BA3
:10DB300053F82500F8BD00BF38120100B4F8FF1FEC
:10DB400070B50B4C2218054692F800260E465AB9BD
:10DB50006C21FFF78BFF06F00F0320F00F021A4332
:10DB60006C212846FFF73EFF631983F8036670BDFA
:10DB7000B4F8FF1F38B50C466C210546FFF776FF59
:10DB8000240104F0700420F07002224328466C2126
:10DB9000BDE83840FFF726BF38B50C466C21054676
:10DBA000FFF764FFE40304F4C03420F4C0322243DE
:10DBB00028466C21BDE83840FFF714BF38B50C4645
:10DBC0006C210546FFF752FF240504F4700420F48D
:10DBD0007002224328466C21BDE83840FFF702BF9F
:10DBE00038B50C466C210546FFF740FF240604F0CB
:10DBF000706420F07062224328466C21BDE83840F2
:10DC0000FFF7F0BE38B50D466C210446FFF72EFF36
:10DC10003DB140F0804220466C21BDE83840FFF71E
:10DC2000E1BE20F08042F6E738B50D466C2104468F
:10DC3000FFF71CFF3DB140F4002220466C21BDE8F7
:10DC40003840FFF7CFBE20F40022F6E738B50D4686
:10DC50006C210446FFF70AFF3DB140F480222046C4
:10DC60006C21BDE83840FFF7BDBE20F48022F6E706
:10DC700038B50D466C210446FFF7F8FE3DB140F47F
:10DC8000804220466C21BDE83840FFF7ABBE20F44F
:10DC90008042F6E738B50D466C210446FFF7E6FEF4
:10DCA0003DB140F4005220466C21BDE83840FFF7FA
:10DCB00099BE20F40052F6E738B50D466C210446B3
:10DCC000FFF7D4FE3DB140F4805220466C21BDE800
:10DCD0003840FFF787BE20F48052F6E738B50C468F
:10DCE0006C210546FFF7C2FE230748BF20F07000F5
:10DCF0004FEA04124CBF40F4006020F4076002F0C9
:10DD0000700202436C212846BDE83840FFF76ABE26
:10DD100038B50C466C210546FFF7A8FEE40104F473
:10DD2000F06420F4F062224328466C21BDE83840BC
:10DD3000FFF758BEFFF7ECBF38B50D466C2104461F
:10DD4000FFF794FE3DB140F4003220466C21BDE85F
:10DD50003840FFF747BE20F40032F6E708B5074B1E
:10DD6000034493F800262AB96C21FFF77FFE00F0E8
:10DD70000F0008BD93F8030608BD00BFB4F8FF1FED
:10DD800008B56C21FFF772FEC0F3021008BD08B59C
:10DD90006C21FFF76BFEC0F3C13008BD08B56C21E4
:10DDA000FFF764FEC0F3035008BD08B56C21FFF710
:10DDB0005DFEC0F3036008BD08B56C21FFF756FE99
:10DDC000C0F3807008BD08B56C21FFF74FFEC0F3AB
:10DDD000C04008BD08B56C21FFF748FEC0F3804085
:10DDE00008BD08B56C21FFF741FEC0F3803008BDC7
:10DDF00008B56C21FFF73AFEC0F3403008BD08B506
:10DE00006C21FFF733FEC0F3003008BD08B56C216C
:10DE1000FFF72CFEC0F30213020548BF43F00803CE
:10DE2000184608BD08B56C21FFF720FEC0F3C310EB
:10DE300008BDFFF7F7BF08B56C21FFF717FEC0F369
:10DE4000404008BD38B50C466D210546FFF70EFE73
:10DE5000640104F0600420F06002224328466D2132
:10DE6000BDE83840FFF7BEBD38B50C466D2105460C
:10DE7000FFF7FCFD640304F4C04420F4C0422243D5
:10DE800028466D21BDE83840FFF7ACBD38B50C46DB
:10DE90006D210546FFF7EAFD240204F4706420F4C6
:10DEA0007062224328466D21BDE83840FFF79ABDD5
:10DEB00038B50C466D210546FFF7D8FD04F00F0478
:10DEC00020F00F02224328466D21BDE83840FFF7BD
:10DED00089BD38B50D466D210446FFF7C7FD20F416
:10DEE0007F0040EA05426D212046BDE83840FFF73B
:10DEF00079BD38B50D466D210446FFF7B7FD3DB13C
:10DF000040F4004220466D21BDE83840FFF76ABD6D
:10DF100020F40042F6E738B50D466D210446FFF7C0
:10DF2000A5FD3DB140F0807220466D21BDE838402E
:10DF3000FFF758BD20F08072F6E708B56D21FFF7B6
:10DF400095FDC0F3411008BD08B56D21FFF78EFDAA
:10DF5000C0F3413008BD08B56D21FFF787FDC0F360
:10DF6000032008BD08B56D21FFF780FD00F00F000C
:10DF700008BD08B56D21FFF779FD0314D8B21B0663
:10DF800048BF60F0FF0008BD08B56D21FFF76EFDCA
:10DF9000C0F3C03008BD08B56D21FFF767FDC0F3C1
:10DFA000006008BD38B50C4670210546FFF75EFDE0
:10DFB00004F0030420F4401242EA0452284670217F
:10DFC000BDE83840FFF70EBD38B50D467021044658
:10DFD000FFF74CFD3DB140F4002220467021BDE822
:10DFE0003840FFF7FFBC20F40022F6E738B50D46B5
:10DFF00070210446FFF73AFD3DB140F480222046EF
:10E000007021BDE83840FFF7EDBC20F48022F6E730
:10E0100038B50C4670210546FFF728FD04F00304CF
:10E0200020F4403242EA044228467021BDE83840DC
:10E03000FFF7D8BC38B50D4670210446FFF716FD32
:10E0400020F47F4040EA052270212046BDE8384098
:10E05000FFF7C8BC38B50D4670210446FFF706FD32
:10E0600020F0FF0045EA000270212046BDE838405C
:10E07000FFF7B8BC08B57021FFF7F8FCC0F30150FA
:10E0800008BD08B57021FFF7F1FCC0F3C04008BD22
:10E0900008B57021FFF7EAFCC0F3804008BD08B561
:10E0A0007021FFF7E3FCC0F3014008BD08B5702103
:10E0B000FFF7DCFCC0F3072008BD08B57021FFF7AF
:10E0C000D5FCC0B208BD70B50E466F2115461C4682
:10E0D000FFF7CCFC16B1C0F30903336015B1C0F3F0
:10E0E00004432B700CB1000E207070BD2DE9F74376
:10E0F000FAF7C2FA0446FAF7BFFA001B0028B8BFC5
:10E1000040420928F7DD384F0025A946A7F103084A
:10E11000ECB2002211462046FFF764FC0222552390
:10E120008DE80C006C21012300222046FFF708FC3B
:10E1300001260F238DE848000022072310212046E6
:10E14000FFF7FEFB294A70212046FFF74BFC2046D3
:10E15000FFF704FE05F8089078550022202120469C
:10E16000FFF740FC00222D212046FFF73BFC002258
:10E1700021212046FFF736FC324623212046FFF7B7
:10E1800031FCDC2224212046FFF72CFC46F6DB0282
:10E1900025212046FFF726FC40F2B7122621204613
:10E1A000FFF720FC4DF2B71227212046FFF71AFC9B
:10E1B00040F2B71228212046FFF714FCDC222A2166
:10E1C0002046FFF70FFC0A222B212046FFF70AFC0E
:10E1D0003544074A14212046FFF704FC032D97D14C
:10E1E00003B0BDE8F08300BFB7FEFF1F8004050049
:10E1F000FFFF0F0038B5074C044494F8001641B9EE
:10E2000094F80356FFF79CFC012384F8003684F849
:10E21000035638BDB4F8FF1F064B034493F800269D
:10E2200032B1002293F8031683F80026FFF788BC6A
:10E23000704700BFB4F8FF1F0D4B37B501251D54C3
:10E240000C4BC4B21D54002220462721FFF7CAFB05
:10E2500020464FF6FF722621FFF7C4FB00230195ED
:10E2600000931A4620212046FFF76AFB03B030BD19
:10E270004F030020D4040020012809D003D3022832
:10E280000BD000207047074B1869C0F380507047CF
:10E29000044B1869C0F340507047024B1869C0F333
:10E2A0000050704740F00F40002808B50FDB02F027
:10E2B00093F90DA3D3E9002302F01EFB41EC100BF0
:10E2C00002F0F2FE51EC100B02F086FC08BD02F0E9
:10E2D00083F905A3D3E9002302F00EFB41EC100BF8
:10E2E00002F04EFEEEE700BF34F7FFFF7F84EE3F03
:10E2F00008B502F071F908A3D3E9002302F0FCFA93
:10E3000041EC100B02F0D0FE51EC100B02F064FC5B
:10E3100008BD00BFAFF30080EB1100A2941A5D406E
:10E32000002808B50FDB02F057F90DA3D3E900234D
:10E3300002F0B8F941EC100B02F022FE51EC100B88
:10E3400002F04AFC08BD02F047F905A3D3E9002317
:10E3500002F0A8F941EC100B02F0A6FEEEE700BFB8
:10E3600034F7FFFF7F84EE3F07EE900AF8EEE77A7E
:10E3700008B517EE900A02F041F907A3D3E900238C
:10E3800002F090F941EC100B02F0FAFD51EC100B89
:10E3900002F022FC08BD00BFEB1100A2941A5D4000
:10E3A000704700BFFEE74FF0E0210B4A0B4BC1F86E
:10E3B000083D4CF22053D3814DF62813D3811388A6
:10E3C00023F001031B041B0C1380D1F8883D43F498
:10E3D0007003C1F8883D70470020054000800000B0
:10E3E000802800F01F014FF001030F4A04DD8B402D
:10E3F000C2F88C31D3607047402804DD8B40C2F8EE
:10E40000883193607047202804DD8B40C2F8843146
:10E4100053607047404200F01F0058BF41428B409C
:10E42000C2F880311360704700E100E0802800F0FE
:10E430001F024FF001030D4903DD9340C1F88C30FA
:10E440007047402803DD9340C1F88830704720288A
:10E4500003DD9340C1F884307047404200F01F0054
:10E4600058BF42429340C1F88030704700E100E05D
:10E47000074B1A78D2B2012A02D1222903D15A704D
:10E4800001225A7070472129FAD10022F7E700BF14
:10E49000BAFEFF1F70B5154611B91B4B197070BD40
:10E4A000022903D1184B01221A7070BD04291AD118
:10E4B000154B5B78012B25D19488402C28BF402434
:10E4C00000235E1CDBB2A34207D300231A460221BD
:10E4D0001846BDE8704000F047BF2A68D05C00F0E5
:10E4E000C3F83346EDE7032906D1074A5378012BD9
:10E4F00008D100239370E9E7052901BF024B0022F0
:10E500001A705A7070BD00BFBAFEFF1F10B50446E6
:10E51000204600F0C1F80028FAD110BD704738B588
:10E520000A4C012502460B4600202946A57000F042
:10E53000F5FA224618B10023A370122038BD937853
:10E5400003F0FF00002BFAD138BD00BFBAFEFF1F59
:10E55000F8B506460F4600F0F4FC0E4B1A78012A77
:10E5600016D15B78012B13D100F000F988B100259A
:10E57000ECB2A74205D821463046BDE8F840FFF787
:10E58000CEBF301900F0D6F801350028F0D0F2E700
:10E590000C20F8BDBAFEFF1F08B540210248FFF766
:10E5A000D7FF00F095F808BDBDFEFF1F38B5054642
:10E5B00000F0A8F80B28044609D140210548FFF7D0
:10E5C000C7FF28B92846BDE8384000F09BB80024B2
:10E5D000204638BDFDFEFF1F70B50C46461E0025C7
:10E5E0000CB9284670BD16F8010FFFF7DFFF013C9C
:10E5F000002818BF0B25A4B2F2E738B5451E002449
:10E6000015F8010F08B9204638BDFFF7CFFF0028E5
:10E6100018BF0B24F4E707B5012300220093064935
:10E62000064B104600F020FA002814BF1B200020E3
:10E6300003B05DF804FB00BF95E4000071E4000046
:10E6400038B50C46054600F097F8A0420AD32C4492
:10E650000020A54207D000B138BD15F8010B00F02D
:10E6600051F8F6E70B2038BD10B50A4A1178402959
:10E670000ED05378D4180133DBB2402BA07001F1D7
:10E6800001014FF00000117014BF5370507010BDA5
:10E690000B2010BD3DFFFF1F10B50C4A117891B142
:10E6A00092F84230D4180133DBB2A4780470402BC6
:10E6B0004FF0000001F1FF31117014BF82F84230B9
:10E6C00082F8420010BD0A2010BD00BF3DFFFF1FB1
:10E6D000014B1878704700BF3DFFFF1F024B1878B1
:10E6E000C0F14000C0B270473DFFFF1F034B002246
:10E6F0005A7083F842201A70704700BF3DFFFF1F19
:10E70000FFF7F4BF10B50A4A117840290ED05378AC
:10E71000D4180133DBB2402BA07001F101014FF09E
:10E720000000117014BF5370507010BD0B2010BD4D
:10E7300080FFFF1F10B50C4A117891B192F842305A
:10E74000D4180133DBB2A4780470402B4FF00000E2
:10E7500001F1FF31117014BF82F8423082F842009B
:10E7600010BD0A2010BD00BF80FFFF1F014B1878AD
:10E77000704700BF80FFFF1F024B1878C0F14000B8
:10E78000C0B2704780FFFF1F034B00225A7083F80E
:10E7900042201A70704700BF80FFFF1FFFF7F4BFD1
:10E7A00070B50546007801F093F902780023D9B2DC
:10E7B000914207D25C1C03EB830303445E786B78C1
:10E7C0009E4227D1174C2B7A342202FB0142D67885
:10E7D00013B334234B43E218907886420CD000F0F8
:10E7E000030204330C2010FB02302118205C0B893B
:10E7F0004A68497800F090FBD4F89C3083B12A46EF
:10E80000287812F8081F00290CBF03210521BDE854
:10E81000704018472346CAE7937801339370D8E7CE
:10E8200070BD00BFC4FFFF1F2DE9F04F85B00D463E
:10E8300090468DF80F0001F04BF9022D064647D1A6
:10E84000077800235C1CDBB2BB4210DB4FF00009F1
:10E85000DFF8B0B0CA465FFA89F4A74212DC284B51
:10E86000D3F89C30002B45D105B0BDE8F08F03EB09
:10E87000830333440DF10F00DA78597801F0E2F99F
:10E880002346DFE704EB84043444E378A28861780C
:10E89000CDF804A0A07800900DF10F0001F0B0F9C0
:10E8A000A378032B05D15A4661789DF80F0001F03B
:10E8B00031FA6178E37841F0100141EAC311002296
:10E8C000C9B20DF10F0001F0EDF909F10109C2E73C
:10E8D000002DC4D10A490378342000FB03138A1C9D
:10E8E0003633294634329A42B9D002F8341C02F841
:10E8F000331CF7E7424629469DF80F009847B3E7D7
:10E90000C4FFFF1FA1E70000F0B40C7804F060041E
:10E91000202C1D4632D14C78042C1DD00AD8012C55
:10E9200004D003D3022C20D0032C12D00020288046
:10E93000F0BC7047212C1BD004D8202CF6D1F0BCA1
:10E9400000F040B9222C16D0232CEFD1F0BC00F0FF
:10E9500049B9F0BC00F049B902241C8014680025B4
:10E9600025701468671C17606570F0BC00F056B91C
:10E97000F0BC00F01FB9F0BC00F076B9402C06D115
:10E98000044CD4F8A04014B1A446F0BC6047CD209C
:10E99000CEE700BFC4FFFF1F73B50446007801F047
:10E9A00097F863680093A27A637A43EA0223ADF88A
:10E9B000043002780023D9B2914207D25D1C03EBE8
:10E9C000830303445E7863789E4225D1174D237AF2
:10E9D000342202FB0152D67803B334234B43EA18A6
:10E9E000907886420CD000F0030204330C2010FB18
:10E9F00002302918285C0B894A68497800F08CFAA3
:10EA0000D5F89C3033B1227A20785AB104F108024B
:10EA10000521984702B070BD2B46CCE793780133AF
:10EA20009370DAE76A460321F3E700BFC4FFFF1FD4
:10EA300007B543680093437A817A43EA0123ADF82E
:10EA40000430084BD3F89C3002462BB1017A007891
:10EA500029B108320521984703B05DF804FB6A46E6
:10EA60000421F8E7C4FFFF1F2DE9F84305460F46D0
:10EA70001646984601F02CF802789DF820300132B5
:10EA80008146D2B20021284601F09EF80446E8B93A
:10EA9000164A1749284600F086F999F80000154BE8
:10EAA000342200FB022209F101011A449946343351
:10EAB000934201F105010CD14146284600F074F85B
:10EAC000044618B9C9F89C70C9F8A0602046BDE892
:10EAD000F88311F8050C03F8340C11F8040C03F852
:10EAE000330C03F8324C03F8314CE0E709E900003D
:10EAF00029E80000C4FFFF1F08B5074B0022C3F838
:10EB00009C20C3F8A02000F0A1F918B9BDE8084086
:10EB100001F06EB808BD00BFC4FFFF1F2DE9F04132
:10EB2000984605460E46174600F0D2FF04780023AB
:10EB3000D9B2A14207D2013303EB8302024412F897
:10EB4000042CB242F4D1174C34234B43E218D07852
:10EB500092F802E0A0EB0E01C9B2042902D1C12053
:10EB6000BDE8F08100F003010130C0B24FF00C0CA1
:10EB70000CFB0133D070A0EB0E001C44C0B2012886
:10EB800025716671A760A4F80C8007D143463A4608
:10EB900031462846BDE8F04100F0BEB90020BDE88E
:10EBA000F08100BFC4FFFF1F014B002019607047B8
:10EBB00068000020024B0979197100F08DBF00BF79
:10EBC0006800002013B5002402AA1C80044B42F800
:10EBD000041D0979197100F08DFF02B010BD00BF4E
:10EBE0006800002000201880704730B40C460221D5
:10EBF000198021796488084D012C297102D130BC1B
:10EC000000F08EBF022C02D130BC00F095BF002076
:10EC1000188030BC704700BF6800002030B40C463C
:10EC20000221198021796488074D012C297102D1B4
:10EC300030BC00F08DBF022C02D130BC00F09ABF76
:10EC40000020188030BC704768000020044B054A43
:10EC500019795B791171137203210A23FFF75EBFE3
:10EC6000680000204C80FF1FF8B500271F808B78BC
:10EC70000B4CA371C3F340035A0063F30002064632
:10EC80006271FFF7E3FF256845B1A37913F0020233
:10EC90001ABF3A46222121213046A8470020F8BD5C
:10ECA00068000020034B00F108021B680078052172
:10ECB000184700BF7000002070B5094D04462A1D9A
:10ECC000012100F0D7FF80220121204600F0EAFF59
:10ECD0002B68207800220A21BDE87040184700BF49
:10ECE0007000002037B501210DF10702044600F045
:10ECF000C1FF9DF80730074D802B04D12A790121EF
:10ED0000204600F0CFFF2B68207800220B21984787
:10ED100003B030BD70000020436805215A7800F030
:10ED2000C1BF73B50122002405460126002100F071
:10ED300089FF334621468DE850001022284600F016
:10ED40005FFF22462146284600F07CFF23462146ED
:10ED50008DE850001022284600F052FF3146022272
:10ED6000284600F09FFF32460621284600F09AFF11
:10ED700022469021284600F095FF044B28781B6816
:10ED80002246214602B0BDE87040184770000020BE
:10ED900042783AB9C178C90141F0100101F09001FF
:10EDA00000F080BF704773B50C468DF8070001F086
:10EDB0000DFA1F4D2C600446002836D11D4A9DF8DF
:10EDC0000700102100F0A6FF1B4A044612219DF8FF
:10EDD000070000F09FFF194A044314219DF8070023
:10EDE00000F098FFE4B20443154A9DF80700132190
:10EDF00000F090FFE4B20443124A9DF80700172187
:10EE000000F088FF02AEE4B204430F4A16F8010D89
:10EE1000162100F07FFFE4B20443032201213046B3
:10EE200000F040FF0323E4B22B71204602B070BD16
:10EE30007000002023ED000019ED0000B9EC000087
:10EE4000E5EC000091ED0000A5EC000037B502AD47
:10EE5000174B05F8010D0022102128461A6000F01A
:10EE60005BFF12210446284600F056FF142104439C
:10EE7000284600F051FFE4B204431321284600F075
:10EE80004BFFE4B204431721284600F045FFE4B2EB
:10EE900004431621284600F03FFFE4B2204310F05F
:10EEA000FF0003D19DF8070001F09CF903B030BDCD
:10EEB000700000201FB501218DF807000DF10E0232
:10EEC0000DF1070000F0D6FE0DF10F0206210DF145
:10EED000070000F0CFFE9DF80E30802B18D19DF872
:10EEE0000F309B0714D59DF8070000F0EFFD0128B7
:10EEF00004460DD172B60DF1070000F029FB002287
:10EF000021460DF107008DF80E2000F0CBFE62B611
:10EF10009DF80E0004B010BD73B50C4615461E4694
:10EF20008DF80700FFF7C6FF802808D033462A4631
:10EF300021460DF1070000F0A7FA02B070BD0020D5
:10EF4000FBE77047062812D880000129C0B201D122
:10EF50000230C0B2074AC0F34703122101FB03236A
:10EF60001A884FF6FF739A4208BFFF207047FF20B0
:10EF7000704700BF780000202DE9F041314C324D40
:10EF8000324E4FF0000884F800814FF4107285F87B
:10EF900040020F462846FF2101F0BCFE4FF480627C
:10EFA00041463046C5F8446201F0B4FE94F80C3195
:10EFB00043F0800384F80C3194F80C311B06FBD429
:10EFC000234BFF221A7094F80C3143F0400384F86D
:10EFD0000C31204B196897B341F000411960194B6F
:10EFE000310AC6F3074201F0FE0183F89C1083F852
:10EFF000B020320E83F8B420174AC5F848221022F8
:10F0000083F80821012283F89420BF2283F880200E
:10F0100093F8002102F07F0283F8002193F8842006
:10F0200042F0010283F8842093F8842042F0100219
:10F0300083F8842084221A770020BDE8F08121F033
:10F040000041CBE70020074078000020000C0020A2
:10F050005680FF1F00700440000E00200D4B93F8F7
:10F060000C2102F0BF0283F80C21BF2283F880201C
:10F0700093F8842002F0FE0283F8842093F8942011
:10F0800002F0FE0283F894201A7F02F07B021A77C6
:10F090000020704700200740F7B5082304248DE8BE
:10F0A0001800B1F803300D788878B3F5007F81BF80
:10F0B0000023CB7002230B71062D71D8AB00DCB29C
:10F0C000012804BF0234E4B24FEA540E354C122733
:10F0D00007FB0E474FF6FF76B7F800C0B4455FD187
:10F0E0004E78032E5CD801285AD897F80FC0BCF18F
:10F0F000FF0F04BF4FF0000C87F80FC0B1F803C03A
:10F10000122101FB0EFE04EB0E0743EA4003BA7323
:10F11000FA7B7E7402F0010213435BB2D4F84822FA
:10F12000C7F80220D9B2F9733874D4F8447224F8BD
:10F130000EC01BB207EBC30E81F00101CEF8042014
:10F14000AEF802C04FF0080E07F833E007EBC10E2F
:10F15000CEF80420AEF802C012FA8CF24FF0480E3E
:10F1600007F831E0C4F8482228B917F8332062F0D4
:10F170007F0207F8332002AA02EB80002DB20A4971
:10F1800050F8082C11F82530012E0CBF164642F01D
:10F1900001063343DBB201F82530002003B0F0BD97
:10F1A0009520FBE778000020C0200740084610B5F6
:10F1B0001146FFF7C7FEFF281DD0104B1221C0F3E8
:10F1C000470001FB0030D3F84422C37B1CB283F01C
:10F1D000010312F8341001F07F0102F8341012F824
:10F1E000331001F07F0102F833104FF0FF338372C8
:10F1F000C372002010BDC42010BD00BF78000020E5
:10F2000073B50C468DF80700114620461646FFF7E9
:10F2100099FEFF28054620D0214632460DF1070011
:10F22000FFF7C4FFC5F3470312210D4D59436B1877
:10F23000D5F848221888121AC5F8482224B2094A7B
:10F24000002002F824004FF0FF326A549A705A707E
:10F25000DA701A715A7102B070BD9620FBE700BFD8
:10F2600078000020C02007402DE9F0410E4680467E
:10F27000114630461746FFF765FE0C4DC0F34700B8
:10F28000122303FB0050C47BFF2C0DD03A463146BD
:10F290004046FFF78BFF24B2D5F8442212F83430F1
:10F2A00063F07B0302F83430BDE8F0817800002081
:10F2B00010B5084600211446FFF744FE084AC0F383
:10F2C0004700122101FB0020D2F84432C27B03EB3D
:10F2D000C2035A68136823605368636010BD00BF9F
:10F2E0007800002010B50C4620461146FFF72AFE94
:10F2F000FF281AD024B2104B13F82430DBB213F0DD
:10F300000C0F12D09B0712D40C4BD3F8443213F8D5
:10F310003020D2090DD180F00100C0B213F8303096
:10F32000DB0914BF0320002010BD052010BD012003
:10F3300010BD032010BD00BFC02007407800002092
:10F3400008B5FFF7FFFD074A1223C0F3470003FB90
:10F350000020C37BFF2B1EBFD2F84422002102F8FD
:10F36000331008BD780000202DE9F0410846002147
:10F3700090461F46FFF7E6FD2249C0F347001224DE
:10F3800004FB0014E57BFF2D39D022884FF6FF7077
:10F3900093B2834233D0D1F8441285F0010011F9C1
:10F3A000300000282BDB2EB287B901EBC6033846AC
:10F3B0005A80D4F802205A6011F8352002F0400239
:10F3C00062F0770201F83620BDE8F08101EBC60259
:10F3D000BB424FF0000028BF3B466781C4F806805F
:10F3E000207360735380C2F8048011F8353003F045
:10F3F000400363F0770301F83630BDE8F0819420D4
:10F40000BDE8F081780000202DE9F0410C46064669
:10F41000114620461546FFF795FD194BC0F34700EE
:10F42000122202FB003090F80FE0BEF1FF0F24D053
:10F4300027B2144A6CB1407C012D0CBF1421182155
:10F44000012818BF41F0010112F82700014302F81A
:10F45000271012F827106FF3410102F82710D3F894
:10F460004432002203F83E203DB92B462A4621466D
:10F470003046BDE8F041FFF777BFBDE8F08100BF3F
:10F4800078000020C02007402DE9F0410C462046BE
:10F49000012117469846FFF755FDFF2836D01C4B33
:10F4A000C0F34700122202FB0030D3F8446290F808
:10F4B0000FE016F93E30002B28DB23B2154A12F874
:10F4C000235015F0020521D10188C0F806701FFAFB
:10F4D00088F242818A42D8BF11460FFA8EF206EBBB
:10F4E000C2030573457359805F602CB9C82306F8C1
:10F4F00032302046BDE8F08116F83E3003F040037C
:10F5000063F0770306F832302C46F2E79324F0E7F5
:10F5100078000020C0200740034B044883F898106F
:10F520000122114600F0BEBB00200740B8020020B7
:10F53000054B0648002283F89420802283F80C2192
:10F540000121FF2200F0AEBB00200740B8020020DE
:10F5500038B51A4C94F8002102F07F0284F800219B
:10F5600094F80C2102F0DF0284F80C2194F880203A
:10F5700042F0200284F8802094F8842002F0DF0218
:10F5800084F8842094F8942002F0DF0284F8942018
:10F5900094F8942042F0040284F8942044F6206504
:10F5A000013DADB200F0BCFE002DF9D194F89430CD
:10F5B00003F0FB0384F8943038BD00BF00200740FF
:10F5C0002DE9F04FD84DD94C95F8807095F88430DE
:10F5D00095F8906087B0FF221F4094F840328DF874
:10F5E00009208DF80C308DF80D20002301210DF13C
:10F5F000090204F510708DF80E3004938DF8153063
:10F600008DF816308DF80F308DF8143000F032FB85
:10F6100095F80C31D907F6B20FD59DF80930802B3B
:10F620000BD195F8003103F07F0385F8003195F890
:10F630000C3103F0DF0385F80C317A0711D5BA4B92
:10F64000042093F8A41093F8A02083F8800006AB60
:10F6500042EA012223F80E2D03A91220049300F0A0
:10F660006DFBFB074BD5B04DB0480123BF2685F895
:10F67000803085F8886095F89430002743F00203C5
:10F6800085F894304FF4107285F89870FF2185F852
:10F69000007101F03FFB4FF480623946D4F8440218
:10F6A00001F038FBD4F8443203F50073C4F8483253
:10F6B0009F4BFF221A7095F8943003F0FD0385F8F4
:10F6C000943095F80C3143F0400385F80C319F23BA
:10F6D00085F88C6085F8843095F8943003F0DF036A
:10F6E00085F8943003A9102000F028FB95F8943099
:10F6F00003F0DF0385F8943007B0BDE8F08F3D07D5
:10F7000040F19380884B082283F880203309C6F3A8
:10F71000C000062B8DF80D308DF80F0000F2F4803C
:10F72000C6F3800202EB830208B10232D2B2D4F8EF
:10F73000446206EBC201C2F34705D1F804E04988F0
:10F74000ADF81510122101FB0541CDF810E091F83C
:10F750000FC08CF0010C81F80FC016F8321082F047
:10F76000010A5FFA8AFAC1F380110FFA8AF881F070
:10F770000101890106EBC80906F83810002800F0DD
:10F78000D980DFF8ACB19BB99BF8002082B9FF2289
:10F7900019468BF8002003A81A460193FFF706FDCF
:10F7A000019B06F838301A46194603A8FFF7DCFD1E
:10F7B0009BF80030012B04D09DF80D30002B00F099
:10F7C000AD80122101FB0541BDF815008B894A89E6
:10F7D00003449BB293428B8109D3B1F800E0C0B2DD
:10F7E000864540F09380897B012940F08F8012216B
:10F7F00001FB0544D4F8061020881944D31A83422B
:10F80000D8BF98B2A9F80200C9F8041016F83A3027
:10F8100003F0400363F0770306F83830424A92F869
:10F82000943003F0DF0382F89430B80717D53E4CCC
:10F83000022384F8803094F8883094F88C2003A94F
:10F84000134016208DF8143000F078FABF2384F8A6
:10F85000883094F8943003F0DF0384F89430F9068C
:10F860001CD5314C202384F88030102384F880305C
:10F8700003A9142000F062FA94F80C3143F020033D
:10F8800084F80C3194F8003143F0800384F800319F
:10F8900094F8843043F0200384F88430BA060DD500
:10F8A000214C202384F8803003A9132000F046FA6D
:10F8B00094F8843003F0DF0384F884303B067FF54E
:10F8C0001BAF0DF10A02FF23102103A88DF80D30A4
:10F8D00000F0D0F99DF80A30134C012B04BF8DF8CD
:10F8E0000F3000224FF0800308BF8DF80D2003A9D0
:10F8F00084F88030172000F021FA94F8943003F057
:10F90000DF0384F89430F7E6FF2210E7122202FBAF
:10F910000544D4F806200492ADF8153003A99DF8EB
:10F920000D0000F00BFA79E7002007407800002076
:10F930005680FF1F6BB916F832202F4902F03C02A7
:10F94000342A35D101238DF80E309EF80030DB09C2
:10F950000B70122101FB05414FF6FF734A899A4251
:10F96000DCD0BDF815E08B8973449BB28B8109888C
:10F970008E4501D19A420CD88AB3B2FBF1F001FB5B
:10F98000102080B258BB122000FB0540807B01286C
:10F9900025D1D21A8A42D8BF91B2122202FB054465
:10F9A000C9B9D4F80230C9F80430A9F802102DE71B
:10F9B0000A78012ACDD1FF200870194603A80193C7
:10F9C000FFF7F4FB019B06F838301A46194603A8E6
:10F9D000FFF7CAFCBDE7D4F806201344E3E7122280
:10F9E00002FB0544D4F80620ADF815304FF0FF3384
:10F9F0000492A372E37291E75680FF1F13460A46F2
:10FA0000194601F087B900BF30B50329039C04985B
:10FA10001DD12BB9164A226004220280002030BD7D
:10FA200040F209418B420FD1022A4FF000030CD85B
:10FA300010490C2505FB0313D9681B6951F82210E6
:10FA400021609B5C0380E9E701230122F0E707299D
:10FA500001D9CD2030BD074B03EB8102126A226031
:10FA6000002AF6D003EB4103B3F84030EAE700BFC9
:10FA70005780FF1FC412010001299FBF034B5B5C2D
:10FA80001370002088BFCD20704700BFC402002043
:10FA900001299DBF024B00205A54CD20704700BF62
:10FAA000C402002019B14B1E584258417047012032
:10FAB0007047054B1A788A4204D05878431A584246
:10FAC0005841704701207047C40200200020704751
:10FAD000004870471413010001299FBF044BC1EB7C
:10FAE000C101C918002094BF1160CD20704700BF2C
:10FAF0005B80FF1F012930B50ED8084DC1EBC10155
:10FB000008231068C45CC818284401330F2B00F880
:10FB1000084CF6D1002030BDCD2030BD5B80FF1FEA
:10FB200001299FBF034B03EB41010020116088BFF7
:10FB3000CD207047C602002001299FBF034B03EB75
:10FB400041010020116088BFCD207047CA0200200B
:10FB500001290AD813681878054B03EB4101887016
:10FB600013685B78CB7000207047CD20704700BFD2
:10FB7000C402002001290AD813681878054B03EB4A
:10FB80004101887113685B78CB7100207047CD20EC
:10FB9000704700BFC4020020084B5A7803F8022BBC
:10FBA000FF210022D1540132072AFBD1044A00234D
:10FBB000052199540133072BFBD17047CE02002059
:10FBC000D702002000BF7047013AD2B2062A10B512
:10FBD0001C4608D8054B5A70FFF7DEFF2146BDE8EA
:10FBE0001040FFF7C9B9992010BD00BFCE02002018
:10FBF000024B00225A70FFF731BA00BFCE0200203C
:10FC000037B50F4C257805B9C1B98DF802308DF89C
:10FC100000109DF81830ADF8032069469DF81C20AF
:10FC200000788DF80130FFF737FA9DF800301BB1EE
:10FC300010B92378013B237003B030BD9520FBE75A
:10FC4000CE02002038B50A4B0D461C7859788C42FC
:10FC50001C4600D14DB929460078FFF7D1FA2DB1E5
:10FC600020B923780133237038BD962038BD00BFFA
:10FC7000CE0200204B1E062B05D8094B19444B78A9
:10FC8000137000207047CB0607D501F00F0106293D
:10FC900003D8034B19444B7AF2E78220704700BF28
:10FCA000CE0200204B1E062B2DE9F0418046174660
:10FCB00005D8174B19444A700020BDE8F081CB06E7
:10FCC00022D501F00F05062D1ED8012A4FEAD114C6
:10FCD0000F4E06D122462946FFF7C6FA35446F7209
:10FCE000EAE7002AFAD173195B7A012BF6D1224692
:10FCF0002946FFF789FB002DF0D184F00102294647
:10FD00004046FFF781FBE9E78220BDE8F08100BFB4
:10FD1000CE02002000207047062903D9A1F110036C
:10FD2000072B07D8044B53F82130002B0CBFC420FD
:10FD300000207047C42070473C130100102810B504
:10FD40000C4601D1FFF728FF034B53F820300BB1CD
:10FD500020469847002010BD3C1301001FB51446F3
:10FD600002228DF807001A8005210DF10F020DF116
:10FD70000700FFF77FFF034B9DF80F201A802360D9
:10FD800004B010BDE00200201FB5144601228DF81A
:10FD900007001A8004210DF10F020DF10700FFF793
:10FDA00069FF044B9DF80F201A800020236004B0E7
:10FDB00010BD00BFE0020020F0B5002685B01E8017
:10FDC00049888DF80700ADF80E10FFF76BFE18B3E9
:10FDD000BDF80E20114F04ACB2FA82F25209012193
:10FDE0000DF10700FFF75EFF34F8022D0421D2B2B7
:10FDF0000DF10700FFF756FF7B68224601210546FB
:10FE00009DF8070098477B689DF80700324602215D
:10FE10009847284605B0F0BD0425FAE7E002002027
:10FE200073B502AC002504F8010D0E461D800422B6
:10FE300001212046FFF736FF7288024B28461A72CE
:10FE400002B070BDE002002013B54C8889888DE8AF
:10FE50000C000B46E2B2210AFFF7D6FD02B010BD3E
:10FE60002DE9F04186B017461E4606AA00238846B3
:10FE7000059303238DF80F0002F8083D01210DF1D1
:10FE80000F00FFF7F7FE98F80050274C15F0030518
:10FE900028D10DF1110206210DF10F00FFF7EAFE46
:10FEA0009DF811309DF80F0003F0030323800DF13E
:10FEB0001203019305AB00932A462B460221FFF75C
:10FEC000A3FD059BDB7913F0400F238814BF43F09B
:10FED000010323F001032380022333803C6006B03A
:10FEE000BDE8F081012D08D19DF81030012B02D121
:10FEF00098F80430ABB90023EDE7022DEED198F865
:10FF0000041041F010010DF11202C9B20DF10F0001
:10FF1000FFF7B0FE9DF8123003F001032380358017
:10FF2000DCE7CD20DAE700BFE00200207FB5002249
:10FF30001A800B784E788DF8070013F003030D46F6
:10FF4000C6F3400634D1FEB14B88013B9BB2012B76
:10FF500052D80DF10F0206210DF10700FFF78AFEBE
:10FF6000044670B9AB7801229A409DF80F301A43CD
:10FF7000D2B206210DF107008DF80F20FFF792FE97
:10FF80000446204604B070BD4E88012E34D10DF1D8
:10FF90000F0206210DF10700FFF76CFE0446002852
:10FFA000EFD1AA7896409DF80F2022EA0602E0E7FA
:10FFB000022B21D109798DF80F10324641F0100142
:10FFC0000DF10700FFF76EFE6B78002E14BF0721BE
:10FFD0000821012B044607D19DF80F00C10900F04C
:10FFE0000F00FFF7ADF90821044B9DF807005B688F
:10FFF0000DF10F029847C4E7CD24C2E7E0020020CC
:020000021000EC
:1000000010B500241C800B7803F00303012B05D1ED
:100010008A780979FFF73CFD204610BD042010BD09
:1000200038B515460A7802F00302012A07D1054CBB
:100030001A8009792246FFF71FFD2C6038BD042085
:1000400038BD00BFE002002013B5CD298DF80700B0
:1000500007D1012290210DF10700FFF723FE02B026
:1000600010BD0D491C88088A1268844288BF188018
:100070000C461B889DF807000021FEF74DFF94F900
:100080000A30002BEBDA00231A4619460DF107005F
:10009000FFF76AF9E3E700BFE002002073B5054609
:1000A00000266A4601218DF800600196FFF7E2FD07
:1000B000AA78434C012A52D168680368C4F80A3010
:1000C0004368A07AC4F80E3004F10A0110F0600F02
:1000D0001ED1E27A3B4B53F82240002C3DD09DF8D4
:1000E0000000022839D802EB42021344034493F87B
:1000F0003430012B31D10DF1020301AA2878A04739
:100100000DF1020301AA01462878FFF79DFF13E0D5
:10011000238AADF80230202B17D87BB102060DD40C
:100120000A68C4F812204A68C4F81620314604F15F
:100130001A022846FFF718F902B070BDE46B64B1EB
:100140000DF1020301AA2049D8E702A82B7800F894
:10015000073D9021FFF7A6FDEEE7CD20D0E79DF803
:100160000030042B10D12B78217A02AD05F8063D22
:100170002846FFF7D1F9012211462846FFF792FDE4
:10018000227A03212846E5E794F90A30002BD3DBD5
:10019000EB78002BD0D1E66B86B1B5F80930287822
:1001A0000833ADF8023004F112010DF1020301AA87
:1001B000B04701460DF1020301AAA5E7CD21F9E7F9
:1001C000E00200209C130100EA020020034B59606A
:1001D000DA630021024AFFF79DBD00BFE002002064
:1001E0009D00010007B502AB054A03F8010D00218F
:1001F00018465160D163FFF78FFD03B05DF804FB33
:10020000E002002000207047354B41F248015A5867
:1002100022F00F0242F002025A5041F204015A58F1
:1002200042F480225A5041F234015A5842F480225A
:100230005A5003F52C33602193F8942042F00202C7
:1002400083F89420C02283F80021FF221A7483F8D7
:10025000802083F8882083F88420002283F88C2073
:1002600083F80C111F491A75080A00F0FE0083F884
:10027000982083F8C02083F8C42083F8C82083F82E
:10028000CC2083F8D02083F8D42083F8D82083F8BA
:10029000DC2083F8E02083F8E42083F8E82083F86A
:1002A000EC2083F8F02083F8F42083F8F82083F81A
:1002B000FC2083F89C00C1F30740090E83F8B000CE
:1002C00083F8B41083F8AC201A7783F8082193F8E8
:1002D000942002F0D40242F0010283F89420704787
:1002E00000700440000C0020024B4FF400125A60D2
:1002F000704700BF00E100E0034B4FF40012C3F869
:1003000084215A60704700BF00E100E008B5FEF7A5
:1003100082F910B9FFF7F0FF08BD1B2008BD00BF30
:10032000034B4AF202629A814BF280429A817047F3
:100330000020054081F0004102E000BF83F000434F
:1003400030B54FEA41044FEA430594EA050F08BF70
:1003500090EA020F1FBF54EA000C55EA020C7FEA34
:10036000645C7FEA655C00F0E2804FEA5454D4EBB1
:100370005555B8BF6D420CDD2C4480EA020281EA7B
:10038000030382EA000083EA010180EA020281EAB3
:100390000303362D88BF30BD11F0004F4FEA013105
:1003A0004FF4801C4CEA113102D0404261EB410114
:1003B00013F0004F4FEA03334CEA133302D052429A
:1003C00063EB430394EA050F00F0A780A4F1010456
:1003D000D5F1200E0DDB02FA0EFC22FA05F2801890
:1003E00041F1000103FA0EF2801843FA05F3594176
:1003F0000EE0A5F120050EF1200E012A03FA0EFCF5
:1004000028BF4CF0020C43FA05F3C01851EBE3711E
:1004100001F0004507D54FF0000EDCF1000C7EEB3B
:1004200000006EEB0101B1F5801F1BD3B1F5001F79
:100430000CD349085FEA30004FEA3C0C04F1010498
:100440004FEA445212F5800F80F09A80BCF1004FC1
:1004500008BF5FEA500C50F1000041EB045141EA43
:10046000050130BD5FEA4C0C404141EB010111F444
:10047000801FA4F10104E9D191F0000F04BF0146EF
:100480000020B1FA81F308BF2033A3F10B03B3F1CD
:1004900020020CDA0C3208DD02F1140CC2F10C025D
:1004A00001FA0CF021FA02F10CE002F11402D8BFBB
:1004B000C2F1200C01FA02F120FA0CFCDCBF41EA87
:1004C0000C019040E41AA2BF01EB0451294330BD56
:1004D0006FEA04041F3C1CDA0C340EDC04F1140433
:1004E000C4F1200220FA04F001FA02F340EA03000A
:1004F00021FA04F345EA030130BDC4F10C04C4F150
:10050000200220FA02F001FA04F340EA030029462F
:1005100030BD21FA04F0294630BD94F0000F83F479
:10052000801306BF81F480110134013D4EE77FEA5C
:10053000645C18BF7FEA655C29D094EA050F08BFA8
:1005400090EA020F05D054EA000C04BF1946104689
:1005500030BD91EA030F1EBF0021002030BD5FEACD
:10056000545C05D14000494128BF41F0004130BDF5
:1005700014F580043CBF01F5801130BD01F0004549
:1005800045F0FE4141F470014FF0000030BD7FEABC
:10059000645C1ABF194610467FEA655C1CBF0B46B7
:1005A000024650EA013406BF52EA033591EA030FCE
:1005B00041F4002130BD00BF90F0000F04BF0021C6
:1005C000704730B54FF4806404F132044FF00005F9
:1005D0004FF0000150E700BF90F0000F04BF002172
:1005E000704730B54FF4806404F1320410F00045D8
:1005F00048BF40424FF000013EE700BF42004FEAD3
:10060000E2014FEA31014FEA02701FBF12F07F434F
:1006100093F07F4F81F06051704792F0000F14BF4C
:1006200093F07F4F704730B54FF4607401F0004590
:1006300021F0004120E700BF50EA010208BF7047E7
:1006400030B54FF000050AE050EA010208BF7047DC
:1006500030B511F0004502D5404261EB41014FF445
:10066000806404F132045FEA915C3FF4DCAE4FF049
:1006700003025FEADC0C18BF03325FEADC0C18BF30
:10068000033202EBDC02C2F1200300FA03FC20FA81
:1006900002F001FA03FE40EA0E0021FA02F11444CE
:1006A000C1E600BF70B54FF0FF0C4CF4E06C1CEAE3
:1006B00011541DBF1CEA135594EA0C0F95EA0C0F58
:1006C00000F0DEF82C4481EA030621EA4C5123EACB
:1006D0004C5350EA013518BF52EA033541F48011FA
:1006E00043F4801338D0A0FB02CE4FF00005E1FBAD
:1006F00002E506F00042E0FB03E54FF00006E1FBF7
:1007000003569CF0000F18BF4EF0010EA4F1FF0439
:10071000B6F5007F64F5407404D25FEA4E0E6D4179
:1007200046EB060642EAC62141EA55514FEAC5208A
:1007300040EA5E504FEACE2EB4F1FD0C88BFBCF506
:10074000E06F1ED8BEF1004F08BF5FEA500E50F1B7
:10075000000041EB045170BD06F0004646EA01017D
:1007600040EA020081EA0301B4EB5C04C2BFD4EBAF
:100770000C0541EA045170BD41F480114FF0000EA8
:10078000013C00F3AB8014F1360FDEBF002001F016
:10079000004170BDC4F10004203C35DA0C341BDC90
:1007A00004F11404C4F1200500FA05F320FA04F062
:1007B00001FA05F240EA020001F0004221F0004196
:1007C00010EBD37021FA04F642EB06015EEA430E09
:1007D00008BF20EAD37070BDC4F10C04C4F1200539
:1007E00000FA04F320FA05F001FA04F240EA0200EC
:1007F00001F0004110EBD37041F100015EEA430EBD
:1008000008BF20EAD37070BDC4F1200500FA05F2DC
:100810004EEA020E20FA04F301FA05F243EA02035B
:1008200021FA04F001F0004121FA04F220EA02006A
:1008300000EBD3705EEA430E08BF20EAD37070BDB0
:1008400094F0000F0FD101F00046400041EB010190
:1008500011F4801F08BF013CF7D041EA060195F072
:10086000000F18BF704703F00046520043EB03032C
:1008700013F4801F08BF013DF7D043EA0603704719
:1008800094EA0C0F0CEA135518BF95EA0C0F0CD024
:1008900050EA410618BF52EA4306D1D181EA03016A
:1008A00001F000414FF0000070BD50EA410606BF64
:1008B0001046194652EA430619D094EA0C0F02D1A9
:1008C00050EA013613D195EA0C0F05D152EA0336EE
:1008D0001CBF104619460AD181EA030101F000410C
:1008E00041F0FE4141F470014FF0000070BD41F055
:1008F000FE4141F4780170BD70B54FF0FF0C4CF42F
:10090000E06C1CEA11541DBF1CEA135594EA0C0F4D
:1009100095EA0C0F00F0A7F8A4EB050481EA030E9A
:1009200052EA03354FEA013100F088804FEA033381
:100930004FF0805545EA131343EA12634FEA02224F
:1009400045EA111545EA10654FEA00260EF0004110
:100950009D4208BF964244F1FD0404F5407402D262
:100960005B084FEA3202B61A65EB03055B084FEAF3
:1009700032024FF480104FF4002CB6EB020E75EBF0
:10098000030E22BFB61A754640EA0C005B084FEA18
:100990003202B6EB020E75EB030E22BFB61A754695
:1009A00040EA5C005B084FEA3202B6EB020E75EBE0
:1009B000030E22BFB61A754640EA9C005B084FEA58
:1009C0003202B6EB020E75EB030E22BFB61A754665
:1009D00040EADC0055EA060E18D04FEA051545EA54
:1009E00016754FEA06164FEAC30343EA52734FEAFD
:1009F000C2025FEA1C1CC0D111F4801F0BD141EA76
:100A000000014FF000004FF0004CB6E711F4801FDA
:100A100004BF01430020B4F1FD0C88BFBCF5E06FBA
:100A20003FF6AFAEB5EB030C04BFB6EB020C5FEACA
:100A3000500C50F1000041EB045170BD0EF0004E1F
:100A40004EEA113114EB5C04C2BFD4EB0C0541EA51
:100A5000045170BD41F480114FF0000E013C90E64E
:100A600045EA060E8DE60CEA135594EA0C0F08BF12
:100A700095EA0C0F3FF43BAF94EA0C0F0AD150EA11
:100A800001347FF434AF95EA0C0F7FF425AF1046A4
:100A900019462CE795EA0C0F06D152EA03353FF4CC
:100AA000FDAE1046194622E750EA410618BF52EA49
:100AB00043067FF4C5AE50EA41047FF40DAF52EA1D
:100AC00043057FF4EBAE12E74FF0FF3C06E000BFBA
:100AD0004FF0010C02E000BF4FF0010C4DF804CDC7
:100AE0004FEA410C7FEA6C5C4FEA430C18BF7FEA87
:100AF0006C5C1BD001B050EA410C0CBF52EA430CB5
:100B000091EA030F02BF90EA020F0020704710F134
:100B1000000F91EA030F58BF994208BF90422CBFC3
:100B2000D8176FEAE37040F0010070474FEA410CBC
:100B30007FEA6C5C02D150EA013C07D14FEA430CDA
:100B40007FEA6C5CD6D152EA033CD3D05DF8040B4B
:100B5000704700BF8446104662468C46194663467D
:100B600000E000BF01B5FFF7B7FF002848BF10F154
:100B7000000F01BD4DF808EDFFF7F4FF0CBF012099
:100B800000205DF808FB00BF4DF808EDFFF7EAFF15
:100B900034BF012000205DF808FB00BF4DF808EDD0
:100BA000FFF7E0FF94BF012000205DF808FB00BFC5
:100BB0004DF808EDFFF7CEFF94BF012000205DF84F
:100BC00008FB00BF4DF808EDFFF7C4FF34BF01205C
:100BD00000205DF808FB00BF4FEA410212F5001249
:100BE00015D211D56FF47873B3EB625212D94FEA74
:100BF000C12343F0004343EA505311F0004F23FA5E
:100C000002F018BF404270474FF00000704750EAB2
:100C1000013005D111F0004008BF6FF0004070476F
:100C20004FF00000704700BFFDF7BDFB002103E05F
:100C30000A4B5B584350043109480A4B42189A4208
:100C4000F6D3094A02E0002313600432074B9A42AC
:100C5000F9D300F00DF88047704700002814010018
:100C60000880FF1F6C85FF1F0086FF1F24100020D7
:100C7000254C08B5F7F705FCF7F76CFCF7F7D2FD44
:100C8000F7F7E4FDF7F7EEFCF7F7CCFFFCF710FD04
:100C9000FCF7F8FAF8F75DF9F7F776FE2078F7F742
:100CA000F1FCE078F7F75EFDF7F717FF28B1F7F7EB
:100CB00014FF6070F7F711FFA060F7F78FFF21892D
:100CC0006079228AFCF738FBFDF710FAFCF788FD03
:100CD0000E4B4FF400725A60FAF7CEFEFBF796FB0C
:100CE0000B4B04225A60FAF7EDFFFBF7D3FBFBF73F
:100CF0008EFBF7F726FFF7F761FF0028F3D0FDF72B
:100D0000F5F9FAF7B9FEEEE70C80FF1F80F00F400F
:100D100000F00F4070B4860746D0541E002A41D020
:100D2000CAB2034602E014F1FF343BD303F8012BAF
:100D30009D07F8D1032C2ED9CDB245EA05250F2CFD
:100D400045EA054519D903F110022646103E0F2E3B
:100D500042F8105C42F80C5C42F8085C42F8045C13
:100D600002F11002F2D8A4F1100222F00F0204F0F6
:100D70000F041032032C13440DD91E462246043AA8
:100D8000032A46F8045BFAD8221F22F00302043239
:100D9000134404F003042CB1C9B21C4403F8011B32
:100DA0009C42FBD170BC704714460346C2E700BFAB
:100DB0002DE9F84355EC104BC5F30A52A2F2FF336C
:100DC000132B064612DC002B41DB244A42FA03F3C4
:100DD00005EA030252EA040017D105F00043024677
:100DE00086ED000B43EC102BBDE8F883332B1CDCA5
:100DF000A2F213424FF0FF3323FA02F214EA020781
:100E00001CD0A94624EA020803E04FF0000825EAB6
:100E1000030942464B4620462946C6E90023FFF710
:100E20008DFA41EC100BBDE8F883002205F0004379
:100E300086ED000B43EC102BBDE8F88305F0004372
:100E40003A4686ED000B43EC102BBDE8F8830022F8
:100E500005F00043C6E90023BDE8F883FFFF0F005B
:100E6000024B13B1024800F005B8704700000000C3
:100E7000810E0100002301461A46184600F01EB8F4
:100E800038B50A4C0A4D641BA4100AD004F1804303
:100E9000013B05EB8305013C55F804399847002CCC
:100EA000F9D1BDE8384000F0B3BA00BF2814010002
:100EB00024140100704700BF704700BF2DE9F843BC
:100EC0002C4D0646286898460F469146FFF7F2FFDC
:100ED000294B1C68D4F84831002B3ED05A681F2A91
:100EE0001CDC02F1010E76B103EB82010124C1F892
:100EF0008890D3F8880194402043022EC3F88801DB
:100F0000C1F8088123D00232C3F804E0286843F80E
:100F10002270FFF7D1FF0020BDE8F883174B0BB319
:100F20004FF4C870AFF300800346D8B1D4F848211D
:100F30000260002141600A46C4F848014FF0010EEA
:100F4000C0F88811C0F88C11002EDCD0CCE7D3F8A3
:100F50008C110C43C3F88C41D5E704F5A673C4F893
:100F60004831BBE72868FFF7A7FF4FF0FF30BDE827
:100F7000F88300BF6885FF1F001401000000000017
:100F800051EC100B2DE9F843C1F30A59A9F2FF35D2
:100F9000132D0C4610EE106A884610EE107A22DCF3
:100FA000002D52DB3E4B43FA05F901EA09030343E6
:100FB0001ED039A3D3E90023FFF7C2F90022002392
:100FC000FFF700FE48B1002C04DD4FF4801343FA14
:100FD00005F5A84428EA0904002723463A4643ECCD
:100FE000102BBDE8F883332D06DDB5F5806F3FD0BB
:100FF00041EC100BBDE8F883A9F213494FF0FF3321
:1010000023FA09F910EA090FF2D023A3D3E9002348
:10101000FFF796F900220023FFF7D4FD0028DCD06B
:10102000002C09DD142D32D00127C5F1340507FA53
:1010300005F5AE1928BFB844444626EA09072346F9
:101040003A4643EC102BBDE8F88313A3D3E9002301
:10105000FFF776F900220023FFF7B4FD0028BCD08B
:10106000002C10DB54EA06070BD000270D4CB4E728
:1010700010EE102A0B46FFF763F941EC100BBDE8A8
:10108000F8833C46A9E700274FF00044A5E704F1A8
:101090000108D1E7AFF300809C7500883CE4377EFF
:1010A000FFFF0F000000F03F51EC100BC1F30A539B
:1010B0002DE9F041A3F2FF35132D0C460F4610EE3B
:1010C000106A1DDC002D43DB3D4B43FA05F801EAB5
:1010D0000803034319D038A3D3E90023FFF730F9FD
:1010E00000220023FFF76EFD20B1002C49DB27EA28
:1010F000080400262346324643EC102BBDE8F0815D
:10110000332D06DDB5F5806F32D041EC100BBDE814
:10111000F081A3F213434FF0FF3828FA03F810EAE6
:10112000080FF2D024A3D3E90023FFF709F9002226
:101130000023FFF747FD0028DCD0002C27DB3C46CE
:1011400026EA08062346324643EC102BBDE8F08120
:1011500019A3D3E90023FFF7F3F800220023FFF7D8
:1011600031FD0028C6D0002C1CDB00263446C1E728
:1011700010EE102A0B46FFF7E3F841EC100BBDE828
:10118000F0814FF4801343FA05F52F44AFE7142D97
:1011900010D00123C5F1340503FA05F5AE1928BFB7
:1011A000FF18CCE724F00042064B324318BF1C4620
:1011B00000269FE70137C2E79C7500883CE4377E34
:1011C000FFFF0F000000F0BF802500004038000046
:1011D000004B0000807000000096000000E100005D
:1011E000002C010000C201000084030090D0030025
:1011F00020A1070040420F0050C3000088130000E8
:10120000018008080000000000000000C800000085
:101210000100C80000800000000000000000000085
:1012200000000000000000000000000000000000BE
:10123000000000000000000001000200040008009F
:10124000100020000101010001000000000000006A
:10125000000000000000010000000000000000008D
:10126000000000000101010000000000000000007B
:101270000001000000000000010101000101000167
:10128000010000000000000000000000000000005D
:10129000000000000000000000000000000000004E
:1012A000000000000000000000000000000001013C
:1012B000010000010001000100000000000000002A
:1012C000000000005780FF1F040000000904000018
:1012D0002813010038130100000000000000000086
:1012E00000000000000000002E81FF1FEB80FF1FA8
:1012F00000000000000000000000000000000000EE
:101300000000000000001200430000000000000088
:10131000000000000301020110000202001000039F
:1013200003011000000100005780FF1FB180FF1F64
:101330008B80FF1F6980FF1F043A26229D00010059
:1013400099E9000031EA0000A1E70000C5FB0000B8
:10135000C5FB0000C5FB0000C5FB0000C5FB00008D
:10136000C5FB0000C5FB0000C5FB0000C5FB00007D
:10137000C5FB0000C5FB0000C5FB000023ED00001D
:10138000B9EC000019ED0000E5EC0000B9EC00003C
:10139000C5FB0000A5EC000091ED000061FE00001F
:1013A0002DFF0000000000002DFF000000000000E5
:1013B00021FE000049FE00000000000089FD000041
:1013C000B9FD000021000100010001005DFD0000E9
:1013D0000101000101000000000101000000000007
:1013E00001010101010000000101000101000100F3
:1013F0000001000001000033323134563130390031
:101400004081FF1FF8B500BFF8BC08BC9E4670477E
:0C141000F8B500BFF8BC08BC9E46704751
:08141C00610E0100358400009F
:04142400118400002F
:10142800F71301000001020000080000010000009D
:1014380002000000000000000000000000000000A2
:101448000000000000000000000000000000000094
:101458000000000000000000000000000000000084
:1014680000000000A1200000000002000000FF04AE
:1014780003090400C2010000000800000000000089
:10148800002203420041004400200053005400524F
:101498000049004E004700200049004E0044004526
:1014A8000058002603530074006500700070006542
:1014B80000720020004D006F0074006F0072002061
:1014C8000044006500760020003A035400520049A9
:1014D800004E0041004D004900430020004D006FC0
:1014E80000740069006F006E00200043006F006EFA
:1014F80000740072006F006C0020002000200020A3
:1015080000200009024300020100C0320904000063
:101518000102020000052400100105240101010454
:1015280024020605240600010705830310000A09A2
:10153800040100020A0000000705810210000007EC
:1015480005020210000012010002020000103C2AED
:101558000001020001020001000000002C84FF1FAE
:101568009484FF1FFC84FF1F00000000000000009F
:101578000000000000000000000000000000000063
:101588000000000000000000000000000000000053
:101598000000000000000000000000000000000043
:1015A8000000000000000000000000000000000033
:1015B8000000000000000000000000000000000023
:1015C8000000000000000000000000000000000013
:1015D8000000000000000000000000000000000003
:1015E80000000000000000000000000000000000F3
:1015F80000000000000000000000000000000000E3
:1016080001000000000000000E33CDAB34126DE67F
:10161800ECDE05000B0000000000000000000000E8
:1016280000000000000000000000000000000000B2
:1016380000000000000000000000000000000000A2
:101648000000000000000000000000000000000092
:101658000000000000000000000000000000000082
:04198800001000202B
:10198C00281401000880FF1F6405000000000000FF
:08199C00000000000000000043
:020000020000FC
:020000041FFFDC
:04800000000000007C
:0400000310000C29B4
:00000001FF
